:100000000C94830C0C94A20C0C94A20C0C94A20CD7
:100010000C94A20C0C94A20C0C94A20C0C94A20CA8
:100020000C94A20C0C94A20C0C94A20C0C94A20C98
:100030000C94A20C0C94A20C0C94A20C0C94A20C88
:100040000C94000F0C94A20C0C94A20C0C94A20C17
:100050000C94D40E0C94A20C0C94A20C0C94A20C34
:100060000C94A20C0C94810F0C94A20C0C94A20C76
:100070000C94A20C0C94A20C0C94A20C0C94A20C48
:100080000C94A20C0C94A20C0C94A20C4C696E65FE
:10009000206E756D626572206F7574206F662072B8
:1000A000616E6765000000000000000000000000B5
:1000B0000000000053796E746178206572726F726F
:1000C0000000000000000000000000000000000030
:1000D000000000000000000000000000496E766192
:1000E0006C69642065787072657373696F6E000067
:1000F0000000000000000000000000000000000000
:1001000000000000556E62616C616E636564207072
:100110006172656E730000000000000000000000C6
:100120000000000000000000000000004461746155
:100130002074797065206D69736D61746368000067
:1001400000000000000000000000000000000000AF
:1001500000000000496C6C6567616C206F7065720F
:1001600061746F72000000000000000000000000D9
:10017000000000000000000000000000496C6C65F9
:1001800067616C207661726961626C6500000000D5
:10019000000000000000000000000000000000005F
:1001A00000000000496C6C6567616C20746F6B65C2
:1001B0006E2028696E7465726E616C206572726F54
:1001C0007229000000000000000000004F7574203C
:1001D0006F66206D656D6F72790000000000000091
:1001E000000000000000000000000000000000000F
:1001F00000000000496E7465676572206F76657255
:10020000666C6F7700000000000000000000000036
:10021000000000000000000000000000496E766150
:100220006C696420686578206469676974000000FF
:1002300000000000000000000000000000000000BE
:1002400000000000486578206E756D626572206F51
:10025000766572666C6F7700000000000000000099
:100260000000000000000000000000004D697373F2
:10027000696E672071756F746500000000000000F2
:10028000000000000000000000000000000000006E
:10029000000000004578706563746564206F7065C8
:1002A0006E206F7220636C6F736520706172656E73
:1002B000000000000000000000000000274F4E2753
:1002C0002073796E746178206572726F720000001D
:1002D000000000000000000000000000000000001E
:1002E000000000004D697373696E67205448454EE5
:1002F00020696E2049462073746174656D656E7463
:100300000000000000000000000000004D69737351
:10031000696E6720544F20696E20464F52207374D7
:100320006174656D656E74000000000000000000DF
:10033000000000004C696E65206E756D626572206C
:100340006572726F72000000000000000000000083
:10035000000000000000000000000000496C6C6517
:1003600067616C20646174612074797065000000BD
:10037000000000000000000000000000000000007D
:100380000000000045787072657373696F6E2074A9
:100390006F6F20636F6D706C657800000000000067
:1003A0000000000000000000000000004D697373B1
:1003B000696E6720636F6D6D6100000000000000D2
:1003C000000000000000000000000000000000002D
:1003D000000000004D697373696E6720636F6D6D77
:1003E00061206F722073656D69636F6C6F6E0000C2
:1003F0000000000000000000000000004D61746873
:1004000020737461636B206F766572666C6F770022
:1004100000000000000000000000000000000000DC
:1004200000000000556E64696D656E73696F6E65DE
:100430006420617272617900000000000000000019
:10044000000000000000000000000000537562730F
:100450006372697074206F7574206F662072616EAC
:1004600067650000000000000000000000000000C0
:1004700000000000446976696465206279207A652D
:10048000726F00000000000000000000000000008B
:100490000000000000000000000000004C696E65D4
:1004A000206E6F7420666F756E640000000000009F
:1004B000000000000000000000000000000000003C
:1004C00000000000546F6F206D616E79206E6573BF
:1004D00074656420474F53554273000000000000CC
:1004E00000000000000000000000000052455455CC
:1004F000524E20776974686F757420474F53554288
:1005000000000000000000000000000000000000EB
:1005100000000000546F6F206D616E79206163747C
:10052000697665205748494C45730000000000007B
:10053000000000000000000000000000454E44578D
:100540004820776974686F7574205748494C450096
:10055000000000000000000000000000000000009B
:10056000000000004F4E20617267756D656E74204B
:100570006D757374206265203E207A65726F00008D
:100580000000000000000000000000004E6F6E73CD
:100590007562736372697074207661726961626CEE
:1005A0006520696E2044494D0000000000000000F5
:1005B000000000005661726961626C6520616C72B6
:1005C000656164792044494D656E73696F6E656439
:1005D000000000000000000000000000546F6F20C9
:1005E0006D616E792061637469766520464F522D86
:1005F0004E455854206C6F6F70730000000000006F
:10060000000000004E45585420646F6573206E6FE3
:1006100074206D6174636820464F52000000000032
:1006200000000000000000000000000043616E2791
:100630007420434F4E54696E756500000000000041
:1006400000000000000000000000000000000000AA
:10065000000000004F7574206F6620646174612093
:10066000696E2052454144206F7220524553544FC9
:100670005245000000000000000000004E65676168
:100680007469766520737562736372697074206E25
:100690006F7420616C6C6F7765640000000000006F
:1006A00000000000496C6C6567616C20454550286E
:1006B0002920617267756D656E740000000000008E
:1006C0000000000000000000000000004F6E6C7988
:1006D00020616C6C6F77656420696E205052494EC2
:1006E000542073746174656D656E740000000000C1
:1006F00000000000417267756D656E74206F75743F
:10070000206F662072616E676520696E20544142D9
:10071000000000000000000000000000546F6F2087
:100720006D616E7920617267756D656E7473206995
:100730006E2043414C4C000000000000000000000F
:1007400000000000417275676D656E7420746F2043
:1007500074696D6524282920697320756E6B6E6F2E
:10076000776E000000000000000000002D2D2034F6
:1007700035202D2D000000000000000000000000CA
:100780000000000000000000000000000000000069
:10079000000000002D2D203436202D2D00000000FB
:1007A0000000000000000000000000000000000049
:1007B0000000000000000000000000002D2D20348B
:1007C00037202D2D00000000000000000000000078
:1007D0000000000000000000000000000000000019
:1007E000000000002D2D203438202D2D00000000A9
:1007F00000000000000000000000000000000000F9
:100800000000000000000000000000002D2D20343A
:1008100039202D2D00000000000000000000000025
:1008200000000000000000000000000000000000C8
:10083000000000002D2D203530202D2D000000005F
:1008400000000000000000000000000000000000A8
:100850000000000000000000000000002D2D2035E9
:1008600031202D2D000000000000000000000000DD
:100870000000000000000000000000000000000078
:10088000000000002D2D203532202D2D000000000D
:100890000000000000000000000000000000000058
:1008A0000000000000000000000000002D2D203599
:1008B00033202D2D0000000000000000000000008B
:1008C0000000000000000000000000000000000028
:1008D000000000002D2D203534202D2D00000000BB
:1008E0000000000000000000000000000000000008
:1008F0000000000000000000000000004E6F7420A7
:10090000656E6F75676820454550524F4D20666F84
:100910007220736176650000000000000000000096
:1009200000000000537461636B20756E646572662D
:100930006C6F770000000000000000000000000065
:100940000000000000000000000000005573657208
:1009500020656E746572656420425245414B00000B
:100960000000000000000000000000000000000087
:100970000000000043616E277420757365204144B8
:100980004452207769746820636F6E7374616E746B
:100990000000000000000000000000004E6F742006
:1009A000656E6F75676820666C61736820666F722C
:1009B0002073617665000000000000000000000068
:1009C0000000000020000000000000000000000007
:1009D0000000000000000000000000000000000017
:1009E00000000000000000000000000000002000E7
:1009F00000000000000000006839636872240000F5
:100A000000000000E3337371727400000000000006
:100A10004B35616273000000000000008633726E87
:100A200064000000000000001C3573676E000000C9
:100A300000000000733974616200000000000000D3
:100A4000000020000000000000000000FC34706581
:100A5000656B000000000000BD346565700000009B
:100A6000000000001C3968657800000000000000EC
:100A70000000200000000000000000005D396865F3
:100A800078320000000000004239686578340000C8
:100A900000000000DF347065656B31360000000037
:100AA000C1347065656B3332000000001935616434
:100AB0006472000000000000B934656570313600D2
:100AC00000000000B534656570333200000000009E
:100AD00000002000000000000000000019386C65D4
:100AE0007400000000000000193800000000000041
:100AF000000000007E397072696E74000000000012
:100B0000B73D666F72000000000000007E3B6E651E
:100B10007874000000000000EB3874726F6E000003
:100B200000000000EF3874726F666600000000007D
:100B3000C936706F6B65000000000000193A6469E7
:100B40006D00000000000000673672656D00000057
:100B50000000000000002000000000000000000075
:100B6000733664617461000000000000413D7265ED
:100B70006164000000000000C33A726573746F7214
:100B8000650000000000676F7375620000000000E0
:100B90000000280000000000000000000000290004
:100BA0000000000000000000C037676F746F000095
:100BB00000000000C8366F6E00000000000000005A
:100BC000B13672657475726E00000000543C69663F
:100BD00000000000000000006F3D696E7075740039
:100BE000000000009C3773746F700000000000006C
:100BF0003937656E64000000000000004C377768EC
:100C0000696C650000000000CA36656E6477680094
:100C100000000000503C656570000000000000000E
:100C20004C3C65657031360000000000483C65654D
:100C300070333200000000000000200000000000BF
:100C40000000000000002000000000000000000084
:100C5000A831616E6400000000000000CA316F72AC
:100C60000000000000000000EC31656F7200000021
:100C7000000000005E3B696E627974650000000050
:100C8000000020000000000000000000B53A6F6E78
:100C900074696D6500000000B63A6F6E697271008C
:100CA00000000000B73A726574690000000000009F
:100CB000B83A6F6E7061636300000000F238736CC5
:100CC00065657000000000000000200000000000CA
:100CD00000000000000020000000000000000000F4
:100CE00000002000000000000000000000002000C4
:100CF00000000000000000000000200000000000D4
:100D000000000000000020000000000000000000C3
:100D1000E8303C000000000000000000BC303E0055
:100D2000000000000000000090303C3D000000008A
:100D30000000000064303E3D0000000000000000A4
:100D400038303D0000000000000000000C303C3E48
:100D50000000000000000000000020000000000073
:100D6000000000000000746F0000000000000000A0
:100D700000007468656E0000000000000000656CF3
:100D800073650000000000000000737465700000CF
:100D90000000000000002000000000000000000033
:100DA0000000200000000000000000000000200003
:100DB0000000000000000000000020000000000013
:100DC0000000000000002000000000000000000003
:100DD00086312B00000000000000000064312D006F
:100DE000000000000000000000002B0000000000D8
:100DF000000000007E393F000000000000000000FD
:100E000067362700000000000000000000002000FE
:100E100000000000000000000000200000000000B2
:100E200000000000000020000000000000000000A2
:100E30000000200000000000000000000000200072
:100E40000000000000000000000020000000000082
:100E50000000000000002000000000000000000072
:100E60000000200000000000000000000000200042
:100E70000000000000000000000020000000000052
:100E80000000000000002000000000000000000042
:100E900014312A00000000000000000015322F006D
:100EA00000000000000000003C316D6F6400000095
:100EB0000000000000002000000000000000000012
:100EC00000002000000000000000000000002000E2
:100ED00000000000000000000000200000000000F2
:100EE00000000000000020000000000000000000E2
:100EF00000002000000000000000000000002000B2
:100F000000000000000000000000200000000000C1
:100F100000000000000020000000000000000000B1
:100F20000000200000000000000000000000200081
:100F30000000000000000000000020000000000091
:100F40000000000000002000000000000000000081
:100F5000A12F5E0000000000000000000000200043
:100F60000000000000000000000020000000000061
:100F70000000000000002000000000000000000051
:100F80000000200000000000000000000000200021
:100F90000000000000000000000020000000000031
:100FA0000000000000002000000000000000000021
:100FB00000002000000000000000000000002000F1
:100FC0000000000000000000000020000000000001
:100FD00000000000000020000000000000000000F1
:100FE00000002000000000000000000000002000C1
:100FF00000000000000000000000200000000000D1
:1010000000000000000020000000000000000000C0
:10101000122F40000000000000000000622F6E6FE1
:1010200074000000000000007F2F2D000000000071
:1010300000000000CA2E4033320000000000000013
:101040003A2F403136000000000000000000200070
:101050000000000000000000000020000000000070
:101060000000000000002000000000000000000060
:1010700000002300000000000000000000003D0010
:101080000000000000000000C0263A000000000040
:101090000000000000003B00000000000000000015
:1010A00000002C00000000000000000000002000F4
:1010B0000000000000000000000020000000000010
:1010C0000000000000002000000000000000000000
:1010D00074696D657230000000000000000000F0CF
:1010E000FF0474696D6572310000000000000000AB
:1010F00000F1FF0474696D657232000000000000A9
:10110000000000F2FF0474696D6572330000000096
:101110000000000000F3FF04665F637075000000CC
:1011200000000000000000F4FF04706F72746100A2
:10113000000000000000000000220001706F7274C7
:101140006200000000000000000000250001706F38
:10115000727463000000000000000000002800011D
:10116000706F727464000000000000000000002B2B
:1011700000016464726100000000000000000000D3
:1011800000210001646472620000000000000000A1
:10119000000000240001646472630000000000008D
:1011A0000000000000270001646472640000000079
:1011B000000000000000002A000170696E6100005C
:1011C00000000000000000000020000170696E6255
:1011D0000000000000000000000000230001706912
:1011E0006E63000000000000000000000026000107
:1011F00070696E640000000000000000000000291B
:10120000000161646373726100000000000000006F
:10121000007A000161646D75780000000000000034
:101220000000007C00016164636C000000000000AD
:1012300000000000007800016164636800000000A5
:1012400000000000000000790001616463000000FC
:10125000000000000000000000780002737073724C
:1012600000000000000000000000004D000173704D
:10127000647200000000000000000000004E000149
:101280007370637200000000000000000000004C5A
:101290000001757074696D650000000000000000B9
:1012A00000FFFF04616463737262000000000000CD
:1012B0000000007B000164696472300000000000DF
:1012C00000000000007E000100000000000000009F
:1012D000000000000000000000000000000000000E
:1012E000000000000000000000000000000A0D6F78
:1012F00072202765652720746F206C6F61642066FB
:10130000726F6D20454550524F4D2E00556E6B6EDD
:101310006F776E20617267756D656E7420746F20D3
:101320004C4F41443B207573652027666C3C6E3EF4
:101330002720746F206C6F61642066726F6D204689
:101340004C41534800206461746120627974657374
:101350002066726F6D20454550524F4D2E00207013
:10136000726F6772616D20627974657320616E645B
:1013700020004C6F616465642000546869732077B5
:10138000696C6C206F766572777269746520746819
:10139000652063757272656E742070726F6772611A
:1013A0006D20696E2052414D2120204172652079C7
:1013B0006F7520737572653F20000A0D4E6F2070A7
:1013C000726F6772616D20736176656420696E204B
:1013D000454550524F4D21002E004E6F20737563CE
:1013E0006820666C6173682066696C653B206D756A
:1013F0007374206265203020746F20002E002064FA
:101400006174612062797465732066726F6D206605
:101410006C6173682066696C6520002070726F676C
:1014200072616D20627974657320616E6420004C76
:101430006F616465642000546869732077696C6C1F
:10144000206F7665727772697465207468652063B1
:10145000757272656E742070726F6772616D212093
:101460002041726520796F7520737572653F200089
:101470000A0D4E6F2070726F6772616D2073617616
:10148000656420696E20666C6173682066696C65AE
:1014900020000A0D6F72202765652720746F207366
:1014A00061766520746F20454550524F4D2E005592
:1014B0006E6B6E6F776E20617267756D656E7420EE
:1014C000746F20534156453B207573652027666C29
:1014D0003C6E3E2720746F207361766520746F2008
:1014E000464C415348004E6F2070726F6772616DB9
:1014F00020696E2052414D3B206E6F7468696E67A3
:101500002073617665642E002064617461206279C5
:1015100074657320746F20454550524F4D2E002046
:1015200070726F6772616D20627974657320616E8D
:1015300064200053617665642000546869732077E5
:10154000696C6C20657261736520746865207072C7
:101550006F6772616D206E6F7720696E2045455010
:10156000524F4D21202041726520796F752073758F
:1015700072653F2000206461746120627974657334
:1015800020746F20666C6173682066696C6520004A
:101590002070726F6772616D20627974657320616B
:1015A0006E64200053617665642000212020417222
:1015B0006520796F7520737572653F2000546869E6
:1015C000732077696C6C206572617365207468653F
:1015D0002070726F6772616D206E6F7720696E2068
:1015E000666C6173682066696C652000206D6172AD
:1015F0006B656420666F72206175746F73746172BD
:10160000742E0050726F6772616D20696E20666C77
:101610006173682066696C6520000A0D4E6F20704A
:10162000726F6772616D20736176656420696E20E8
:10163000666C6173682066696C65200050726F6724
:1016400072616D20696E20454550524F4D206D618D
:10165000726B656420666F72206175746F7374615C
:1016600072742E004E6F2070726F6772616D2073FE
:101670006176656420746F20454550524F4D2100BE
:101680004175746F737461727420666C6167207247
:10169000656D6F7665642E000A0D4B4C426173696F
:1016A0006320666F722041746D656C204156522034
:1016B00041546D65676131323834702076302E3890
:1016C000000A0D436F7265207772697474656E202D
:1016D0006279204B61726C204C756E742C206261B3
:1016E000736564206F6E20476F72646F6E20446F65
:1016F0007567686D616E27732042415349433131EC
:10170000000A0D4B4C426173696320636F72652060
:1017100076302E39000A0D5245414459003A2000D6
:101720004552524F522023005E5E5E003A20002058
:10173000696E206C696E6520004552524F5220231D
:10174000000A0D4E6F2070726F6772616D20696EB6
:10175000206D656D6F72792E000A0D50726F677281
:10176000616D206572617365642E000A0D546869AD
:10177000732077696C6C206572617365207468658D
:101780002063757272656E742070726F6772616D1E
:1017900021202041726520796F7520737572653F35
:1017A00020004E6F2070726F6772616D206C6F61E8
:1017B00064656420696E206D656D6F72792E0A0D07
:1017C000006461746100270072656D004E6F2073C4
:1017D00075636820666C6173682066696C652E00AD
:1017E000204E6F2070726F6772616D2E003A20007C
:1017F000666C0020627974657320667265650044CA
:10180000796E616D6963206D656D6F727920706F9F
:101810006F6C2028617272617973293A200020620E
:1018200079746573206672656500566172696162DC
:101830006C65206D656D6F72793A20002062797455
:10184000657320667265650050726F6772616D2006
:101850006D656D6F72793A2000556E6B6E6F776EA5
:10186000204155544F535420617267756D656E74F5
:101870002E20204D757374206265204F46462C2023
:1018800045452C20464C302C20464C312C206F7284
:1018900020464C322E00496C6C6567616C20617586
:1018A000746F73746172742076616C756520004189
:1018B00075746F73746172742066726F6D20666CDC
:1018C00061736820004175746F737461727420666F
:1018D000726F6D20454550524F4D2E004175746F0B
:1018E0007374617274206E6F7420656E61626C65D2
:1018F000642E000A0D53746F70706564206174204B
:101900006C696E65200011241FBECFEFD0E4DEBFEE
:10191000CDBF13E0A0E0B1E0E6EBFEE700E00BBFD7
:1019200002C007900D92A431B107D9F714E3A4E1E6
:10193000B3E001C01D92A035B107E1F70E94E9179D
:101940000C94593F0C94000028E032E33093C0051A
:101950002093BF053093A3332093A23387E993E309
:101960009093802D80937F2DF90101C01192809179
:101970007F2D9091802D8E179F07C0F786E696E009
:1019800090938B2D80938A2D90937305809372058D
:1019900085E79DE29093792D8093782D08959C01A1
:1019A000220F331FF90143E0EE0FFF1F4A95E1F7C5
:1019B000E20FF31FE152FF4E65917491CB01409607
:1019C000049750F4862F8F7090E0880F991F880F2E
:1019D000991F875E9C4F06C08FEF6F3F780741F4D9
:1019E00085E193E09C01442737FD4095542F0CC0BE
:1019F0008FEF643F780729F420E030E040E050E0CA
:101A000003C09B0140E050E0B901CA0108959C0168
:101A1000285F3D4CC9010895FC01DB0180E29EE294
:101A20009183808388EE93E08D939C930895FC01CD
:101A300010821182128260E070E080E090E00895F0
:101A40000895FC0181E08783838381E090E09187A2
:101A50008087148280E790E09683858360E070E061
:101A600080E090E0089508958091C00085FFFCCF4C
:101A70008DE08093C6008091C00085FFFCCF8AE096
:101A80008093C6000895982F8823C1F18091140394
:101A9000882341F19636E1F0973638F4923681F09A
:101AA000953651F09136A9F40DC0923779F09437FC
:101AB00029F09E3671F408C09BE10BC099E009C083
:101AC00098E007C097E005C09AE003C09DE001C020
:101AD0009CE0109214038091C00085FFFCCF90938E
:101AE000C60008959C3521F481E080931403089585
:101AF0008091C00085FFFCCF9093C6000895CF93DE
:101B0000DF93EC0102C00E94430DFE0121968491F7
:101B10008823C9F7DF91CF91089588E996E10E9463
:101B20007F0D0895CF93DF93EC0102C00E94430D17
:101B300089918823D9F7DF91CF910895982F8091CB
:101B4000C00085FFFCCF9093C60008959091490393
:101B500080914A039817D1F3F894E0914A03F0E09A
:101B6000E75DFC4F808120914A0330E02F5F3F4FBB
:101B70002F71307020934A0378940895FF920F9349
:101B80001F93CF93DF93EC0110E008E060E2F62EA4
:101B90000E94A60D982F8D30A9F488838091C000F3
:101BA00085FFFCCF8AE08093C6008091C00085FF4E
:101BB000FCCF8DE08093C600DF91CF911F910F91F4
:101BC000FF9008958830B9F4112311F38091C0007B
:101BD00085FFFCCF0093C6008091C00085FFFCCF3D
:101BE000F092C6008091C00085FFFCCF0093C60034
:101BF00021971150CDCF8A3059F28091C00085FFD6
:101C0000FCCF9093C60099931F5FC2CF1F93142FF0
:101C1000FC01EE0FFF1F9F0143E0220F331F4A9587
:101C2000E1F7E20FF31FEF51FF4E44919C01220FA9
:101C3000331FF901B3E0EE0FFF1FBA95E1F7E20F92
:101C4000F31FE152FF4EA591B491413011F41C9362
:101C50001CC0423031F4812F952F11969C938E93A6
:101C600014C0CD014096049780F4F894EA2FF0E078
:101C7000EF70F070EE0FFF1FEE0FFF1FE75EFC4FDF
:101C8000108351836283738378941F910895FC01BC
:101C9000EE0FFF1F9F0143E0220F331F4A95E1F72C
:101CA000E20FF31FEF51FF4E44919C01220F331FAF
:101CB000F90183E0EE0FFF1F8A95E1F7E20FF31FB2
:101CC000E152FF4EA591B491413021F48C91282F1F
:101CD00030E005C0423031F48D919C919C0140E090
:101CE00050E030C0CD014096049778F4EA2FF0E040
:101CF000EF70F070EE0FFF1FEE0FFF1FE75EFC4F5F
:101D000020813181428153811DC08FEFAF3FB807E1
:101D100049F4209115033091160340911703509117
:101D2000180310C0A45FBF4F29F020E030E040E06E
:101D300050E008C020915F0330916003409161033F
:101D400050916203B901CA010895833028F020E060
:101D500030E040E050E010C0E82FF0E0EE0FFF1F51
:101D6000EE0FFF1FEE5FFE4F80819181A0E0B0E09B
:101D70002227382F492F5A2FB901CA010895CF932E
:101D8000DF93EC01A0E0B0E009C06BBFFA018791DE
:101D900089934F5F5F4F6F4F7F4F1196A217B30725
:101DA000A0F3DF91CF9108951F920F920FB60F927B
:101DB0000BB60F9211248F939F93EF93FF93809113
:101DC000C600833021F481E08093852D0EC0E09120
:101DD0004903F0E0E75DFC4F80838091490390E088
:101DE00001968F71907080934903FF91EF919F91BD
:101DF0008F910F900BBE0F900FBE0F901F901895F4
:101E00001F920F920FB60F9211248F939F93AF934F
:101E1000BF938091150390911603A0911703B09181
:101E200018030196A11DB11D80931503909316030D
:101E3000A0931703B09318038091190390911A038C
:101E4000A0911B03B0911C030097A105B10559F0A7
:101E50000197A109B1098093190390931A03A093E4
:101E60001B03B0931C0380911D0390911E03A0914E
:101E70001F03B09120030097A105B10559F0019708
:101E8000A109B10980931D0390931E03A0931F0322
:101E9000B09320038091210390912203A09123030A
:101EA000B09124030097A105B10559F00197A1094C
:101EB000B1098093210390932203A0932303B0934D
:101EC00024038091250390912603A0912703B091CC
:101ED00028030097A105B10559F00197A109B1099F
:101EE0008093250390932603A0932703B0932803A0
:101EF000BF91AF919F918F910F900FBE0F901F9048
:101F000018951F920F920FB60F9211240F900FBECB
:101F10000F901F9018959B01BC01660F771FCB0196
:101F2000E3E0880F991FEA95E1F7680F791F605386
:101F30007F4EC9010E941E3F0895CF92DF92EF921B
:101F4000FF920F931F93DF93CF93CDB7DEB72F97F9
:101F50000FB6F894DEBF0FBECDBFFF24A2E1EA2E7C
:101F60006E010894C11CD11CFE9C800111240053F9
:101F70001F4EC8010E94253F892B59F0C601B801A8
:101F80000E941E3FC6010E945B19892BA1F4F394A5
:101F9000EBCF20E030E0C9012F960FB6F894DEBFFA
:101FA0000FBECDBFCF91DF911F910F91FF90EF90AA
:101FB000DF90CF900895E091862DF091872D83E8F2
:101FC0008193F093872DE093862D8F2D90E00E94D2
:101FD000AD1821E030E0DFCFCF93DF930E94671888
:101FE000E0918F2DF091902D808190E0C0970A971D
:101FF00018F0C0E0D0E036C020E030E011C0C901E8
:1020000063E0880F991F6A95E1F7220F331F280FAD
:10201000391F240F351F3196F093902DE0938F2DAB
:10202000E0918F2DF091902D8081482F50E040530A
:1020300050404A30510518F3E9010E946718C33037
:10204000D10584F08AED93E10E947F0D62E070E09B
:1020500080E090E00E946F2188ED93E10E947F0D67
:10206000CFEFDFEFCE01DF91CF9108958F929F9256
:10207000AF92BF92CF92DF92EF92FF920F931F9396
:10208000CF93DF934C01FC01EE0FFF1FEE0FFF1FFC
:10209000E050FF4F80819181A0E0B0E0EE24F82E67
:1020A000092F1A2F7CE0A72EB12CC12CD12CAE0CFD
:1020B000BF1CC01ED11ECBBEF501879196918F5FCC
:1020C0009F4F61F480E794E10E947F0DB40188275F
:1020D00077FD8095982F0E946F2121C120918A2D34
:1020E00030918B2D809172059091730528173907D7
:1020F00089F087E394E10E947F0D8BE493E00E94D6
:10210000BE0D80914B0390E00E940E3F89379105F0
:1021100009F005C1CBBEF501A791B691AA59B94FF7
:10212000B0938B2DA0938A2D4EE050E060E070E0DC
:10213000E40EF51E061F171F0BBFF70147915691BE
:102140004A0F5B1F509373054093720562E070E085
:1021500080E090E0E60EF71E081F191F0BBFF70185
:1021600087919691885F9D4C9093C0058093BF05A1
:1021700062E0A62EB12CC12CD12CEA0CFB1C0C1D4C
:102180001D1D0BBFF70127913691820F931F90936E
:10219000A3338093A23364E070E080E090E0E60E29
:1021A000F71E081F191F0BBFF70187919691805EDC
:1021B000914D9093B8058093B7055A01AA1ABB0AAE
:1021C000F401EE0FFF1FEE0FFF1FEE5FFE4F808149
:1021D00091817C0100E010E0502F4F2D3E2D2227F1
:1021E00060E070E016C04BBFF90187918C932F5FC0
:1021F0003F4F4F4F5F4F222349F40894E11CF11CDD
:10220000011D111D502F4F2D3E2D222711966F5F5E
:102210007F4F6A157B0538F30894E11CF11C011D02
:10222000111D502F4F2D3E2D2227A091BF05B0919B
:10223000C005C090A233D090A333CA1ADB0A60E075
:1022400070E016C04BBFF90187918C932F5F3F4F11
:102250004F4F5F4F222349F40894E11CF11C011DEC
:10226000111D502F4F2D3E2D222711966F5F7F4F4E
:102270006C157D0538F30894E11CF11C011D111D3E
:10228000502F4F2D3E2D2227C091B705D091B80574
:10229000C052DE42A0E2BEE260E070E016C04BBF7A
:1022A000F90187918C932F5F3F4F4F4F5F4F222350
:1022B00049F40894E11CF11C011D111D502F4F2DF4
:1022C0003E2D222711966F5F7F4F6C177D0738F3E5
:1022D0000E947F2D9093A5338093A4338FE294E1E5
:1022E0000E947F0DB50180E090E00E946F218BE19C
:1022F00094E10E947F0DB60180E090E00E946F2182
:102300008EEF93E10E947F0DB401882777FD8095C1
:10231000982F0E946F218CEF93E10E947F0DDF9137
:10232000CF911F910F91FF90EF90DF90CF90BF90D2
:10233000AF909F908F900895EF92FF920F931F930D
:102340007C010E94403F182F00E0C70101960E94C7
:10235000403F080F111DC8011F910F91FF90EF9092
:102360000895AF92BF92CF92DF92EF92FF920F93B8
:102370001F93CF93DF938CE090E00E949C118F5FBE
:102380009F4F19F48AEB93E191C020918A2D3091EF
:102390008B2D80917205909173052817390789F06C
:1023A0008AE793E10E947F0D8BE493E00E94BE0DCB
:1023B00080914B0390E00E940E3F8937910509F010
:1023C00077C08CE090E00E949C11B6E6CB2EB6E080
:1023D000DB2EC80ED91ED0928B2DC0928A2D8EE096
:1023E00090E00E949C117601E80EF91EF0927305B0
:1023F000E092720580E190E00E949C118C01085FE0
:102400001D4C1093C0050093BF0582E190E00E942F
:102410009C11080F191F1093A3330093A233570187
:10242000AC18BD08C0E0D0E008C0CE014A960E94BA
:10243000403FF60181936F012196CA15DB05A8F391
:10244000E090BF05F090C005C090A233D090A333B8
:10245000CE18DF088501065E1F4FC0E0D0E009C03E
:10246000C8010E94403FF70181937F0121960F5FD1
:102470001F4FCC15DD05A0F30E947F2D9093A5334F
:102480008093A43382E793E10E947F0DB50180E041
:1024900090E00E946F218EE593E10E947F0DB601CE
:1024A00080E090E00E946F2185E493E10E947F0D1F
:1024B000DF91CF911F910F91FF90EF90DF90CF9020
:1024C000BF90AF9008950F931F93CF93DF930E9417
:1024D000671800918F2D1091902DF80180818D301B
:1024E00071F090E00E940E3F8536910559F4F80195
:1024F000818190E00E940E3F85369105F1F40E94A3
:10250000B11123C086369105C1F4E8012196F80186
:10251000818190E00E940E3F8C36910571F42196E6
:10252000D093902DC0938F2D0E94EC0FFFEF8F3F23
:102530009F0759F00E94361008C08CE093E10E947A
:102540007F0D8DEE92E10E947F0DDF91CF911F9163
:102550000F91089588E190E00E94403F089588E13E
:1025600090E00E94403F8A3579F08B3518F485352C
:1025700029F407C08B3559F08C3561F020E030E04C
:102580000FC00E94B1110AC080E090E005C081E058
:1025900090E002C082E090E00E94361021E030E03E
:1025A000C9010895CF92DF92EF92FF920F931F938C
:1025B000DC01CB016C010E94403FE82EFF2400E0CB
:1025C00010E0102F0F2DFE2CEE24C60101960E9464
:1025D000403FE80EF11C011D111DB701C8011F91FC
:1025E0000F91FF90EF90DF90CF900895AF92BF9240
:1025F000CF92DF92EF92FF920F931F937B018C019A
:102600000E94D2125B016C016501BB24AA2482E006
:1026100090E0A0E0B0E0E80EF91E0A1F1B1FC80101
:10262000B7010E94D2129B01AC012A0D3B1D4C1D2B
:102630005D1DB901CA011F910F91FF90EF90DF90CE
:10264000CF90BF90AF900895AF92BF92CF92DF929C
:10265000EF92FF920F931F931092490310924A0337
:102660001092852D60E070E080E090E00E94F6120C
:102670007B018C0160935F0370936003809361031F
:102680009093620364E070E080E090E00E94F612B4
:102690005B016C0160936303709364038093650333
:1026A0009093660368E070E080E090E00E94F6128C
:1026B000AE0CBF1CC01ED11EA616B706C806D90692
:1026C000C1F080E09DE2A1E3B1E080935F039093CD
:1026D0006003A0936103B093620380E096E9A0E0F9
:1026E000B0E08093630390936403A0936503B09379
:1026F000660372E0D72ED092C00088E98093C100B3
:1027000086E08093C200E0905F03F0906003009148
:10271000610310916203209163033091640340913F
:1027200065035091660363E0220F331F441F551F5A
:102730006A95D1F7C801B7010E94BD3E21501092A1
:10274000C5002093C400D4BC84E085BDC801B70196
:1027500020E038EE43E050E00E94BD3E215027BD0E
:1027600080916E00826080936E0010921903109227
:102770001A0310921B0310921C0310921D03109257
:102780001E0310921F031092200310922103109237
:102790002203109223031092240310922503109217
:1027A0002603109227031092280378941F910F910B
:1027B000FF90EF90DF90CF90BF90AF900895DC0135
:1027C000CB010E94403F682F70E080E090E00895C8
:1027D0001F93CF93DF93EC01162F0E94403F1817F1
:1027E00021F0CE01612F0E94483FDF91CF911F91D0
:1027F0000895FF920F931F938C01F62E672F0E946E
:10280000E813C80101966F2D0E94E8131F910F91E4
:10281000FF9008958F929F92AF92BF92CF92DF92D6
:10282000EF92FF920F931F93DF93CF93CDB7DEB755
:1028300064970FB6F894DEBF0FBECDBF8CE090E07A
:102840000E949C118F5F9F4F81F08AE395E10E9467
:102850007F0DCE0101960E94BE0D898190E00E94FD
:102860000E3F8937910509F09CC0809172059091C7
:10287000730520918A2D30918B2D821B930B209113
:10288000A2333091A3334091BF055091C005241B62
:10289000350B820F931F4A96875E9F4030F087E387
:1028A00080937A2D0E94E9217CC088E190E06FEF4F
:1028B0000E94E8138CE090E060E070E00E94F91361
:1028C000609172057091730580918A2D90918B2D86
:1028D000681B790B8EE090E00E94F91380E190E094
:1028E00060E070E00E94F9136091A2337091A3330D
:1028F0008091BF059091C005681B790B82E190E043
:102900000E94F913E0908A2DF0908B2D8090720533
:10291000909073058E189F0800E010E009C0C80170
:102920004A96F70161917F010E94E8130F5F1F4FE4
:1029300008151905A0F3C090BF05D090C005A09060
:10294000A233B090A333AC18BD08EAE1EE2EF12C0F
:10295000E80CF91C00E010E00BC0C701F601619122
:102960006F010E94E8130F5F1F4F0894E11CF11CD8
:102970000A151B0590F383E395E10E947F0DB401D6
:1029800080E090E00E946F218FE195E10E947F0D31
:10299000B50180E090E00E946F2188E095E10E94FF
:1029A0007F0D64960FB6F894DEBF0FBECDBFCF91FA
:1029B000DF911F910F91FF90EF90DF90CF90BF902C
:1029C000AF909F908F900895CF92DF92EF92FF92F9
:1029D0000F931F93CF93DF9320918A2D30918B2DEE
:1029E00080917205909173052817390719F486EEC6
:1029F00094E1C7C10E94671800918F2D1091902D0E
:102A0000D8018C918D3079F090E00E940E3F853690
:102A1000910561F4F801818190E00E940E3F8536B6
:102A2000910509F0A8C10E940A14ADC1863691052E
:102A300009F0A1C1E8012196D80111968C9190E08E
:102A40000E940E3F8C36910509F095C12196D093D6
:102A5000902DC0938F2D0E94EC0F6C01BFEF8F3F24
:102A60009B0709F490C1FC01EE0FFF1FEE0FFF1F43
:102A7000E050FF4F80819181A0E0B0E0EE24F82E7D
:102A8000092F1A2F2CE030E040E050E0E20EF31E58
:102A9000041F151F0BBFF7018791969124EF3FEF9D
:102AA0004FEF5FEFE20EF31E041F151F8F5F9F4F66
:102AB000E1F08DEB95E10E947F0DB601882777FD4F
:102AC0008095982F0E946F218BEA95E10E947F0DDF
:102AD0008BE493E00E94BE0D80914B0390E00E9436
:102AE0000E3F8937910509F04EC120917205309152
:102AF000730560918A2D70918B2D922F961B4091BA
:102B0000A2335091A333E091BF05F091C005A42FEB
:102B1000AE1B892F8A0F865E8093932D8FEF809353
:102B20007F03109273031092740390937503261B16
:102B3000370B309376031092770310927803A093AB
:102B400079034E1B5F0B50937A0310927B03109214
:102B50007C038091B7059091B80520E23EE2482FB2
:102B6000421B40937D0380529E42892F990F990BFF
:102B700080937E03C801B70147E653E00E9400FE40
:102B8000F601EE0FFF1FEE0FFF1FEE5FFE4F80817D
:102B900091817C0100E010E0C0E0D0E040E050E036
:102BA0001EC0FA01E959FC4FDE01AA59B94F8C91B8
:102BB00080834F5F5F4F81E04030580779F4902F5A
:102BC0008F2D7E2D662747E653E00E9400FE089475
:102BD000E11CF11C011D111D40E050E02196809187
:102BE00072059091730520918A2D30918B2D821B57
:102BF000930BC817D907A8F2452B41F0902F8F2DC2
:102C00007E2D662747E653E00E9400FE0894E11CF3
:102C1000F11C011D111DC0E0D0E040E050E01EC0DD
:102C2000FA01E959FC4FDE01A85FBD4C8C9180830D
:102C30004F5F5F4F91E04030590779F4902F8F2D0F
:102C40007E2D662747E653E00E9400FE0894E11CB3
:102C5000F11C011D111D40E050E021968091A2332E
:102C60009091A3332091BF053091C005821B930B37
:102C7000C817D907A8F2452B41F0902F8F2D7E2D34
:102C8000662747E653E00E9400FE0894E11CF11C11
:102C9000011D111DC0E0D0E020E030E01EC0F901B0
:102CA000E959FC4FDE01A05EB14D8C9180832F5F0E
:102CB0003F4FA1E020303A0779F4902F8F2D7E2DE1
:102CC000662747E653E00E9400FE0894E11CF11CD1
:102CD000011D111D20E030E021968091B7059091F3
:102CE000B80580529E42C817D907C8F2232B41F07D
:102CF000902F8F2D7E2D662747E653E00E9400FE21
:102D000084EA95E10E947F0D6091720570917305D0
:102D100020918A2D30918B2D621B730B882777FDB4
:102D20008095982F0E946F2180E995E10E947F0D88
:102D30006091A2337091A3332091BF053091C005FB
:102D4000621B730B882777FD8095982F0E946F2157
:102D500085E795E10E947F0DB601882777FD809574
:102D6000982F0E946F218091C00085FFFCCF8EE2DA
:102D70008093C60008C08FEA94E10E947F0D82E92B
:102D800094E10E947F0DDF91CF911F910F91FF90F1
:102D9000EF90DF90CF900895EF92FF920F931F93E3
:102DA0009C018F3F910541F488E190E06FEF0E9414
:102DB000E81380E896E15AC08535910591F48CE0DE
:102DC00090E00E949C118F5F9F4F19F484E696E17A
:102DD0004DC088E190E065E50E94E8138CE396E140
:102DE00045C08A35910511F460E00AC08B35910524
:102DF00011F461E005C08C35910509F039C062E03D
:102E0000E62FF0E0EE0FFF1FEE0FFF1FE050FF4F29
:102E100080819181A0E0B0E0BA2FA92F982F882758
:102E20000C96A11DB11DABBFFC0187919691E62EBA
:102E3000FF2400E010E08F5F9F4F49F48AE196E1A4
:102E40000E947F0DC801B7010E946F2111C088E167
:102E500090E0622F0E94E81383E096E10E947F0DCC
:102E6000C801B7010E946F218CEE95E10E947F0D91
:102E70001F910F91FF90EF900895DF92EF92FF92D4
:102E80000F931F937B018C01D42ECB01652F0E94E1
:102E9000483F0894E11CF11CC7016D2D0E94483F7A
:102EA0001F910F91FF90EF90DF900895AF92BF9226
:102EB000CF92DF92EF92FF920F931F937B018C01D1
:102EC00059016A019A0144275527A9010E943D171B
:102ED00082E090E0A0E0B0E0E80EF91E0A1F1B1FA0
:102EE000C801B701A5010E943D171F910F91FF90E6
:102EF000EF90DF90CF90BF90AF900895DC01CB01B1
:102F0000642F0E94483F08956F927F928F929F9204
:102F1000BF92CF92DF92EF92FF920F931F93DF93B6
:102F2000CF93CDB7DEB72F970FB6F894DEBF0FBEA5
:102F3000CDBF4C01BB2413E1612E712C6E010894AE
:102F4000C11CD11C8B2D90E0869D7001879DF00CDB
:102F5000969DF00C1124870106521D4EC8010E9457
:102F6000253F892BF9F0C601B8010E941E3FC6011A
:102F70000E945B19892BA1F0F701E751FD4E859165
:102F80009591A591B491F40180839183A283B38339
:102F9000F60101900020E9F73197EC19FD0904C012
:102FA000B394D0CFE0E0F0E0CF012F960FB6F894C5
:102FB000DEBF0FBECDBFCF91DF911F910F91FF906C
:102FC000EF90DF90CF90BF909F908F907F906F9009
:102FD00008950E94DC1A81E090E00895FC011182BE
:102FE0004083738362830895FC011182408373835D
:102FF00062830895FC018181882331F460937A2DE6
:103000000E94E92180E00895815081830280F3814C
:10301000E02DE80FF11D80810895DC0111969C914F
:1030200011978C91981729F440937A2D0E94E921E9
:1030300008951296ED91FC911397E90FF11D6083AD
:1030400011968C9111978F5F11968C930895FC01C6
:103050008181882349F460937A2D0E94E92120E040
:1030600030E040E050E010C08150818390E0880F54
:10307000991F880F991F0280F381E02DE80FF91F37
:103080002081318142815381B901CA010895DC0157
:1030900011963C9111978C91381729F420937A2D31
:1030A0000E94E9210895832F90E0880F991F880FCF
:1030B000991F1296ED91FC911397E80FF91F408329
:1030C0005183628373833F5F11963C93089505C0DB
:1030D0003196F093902DE0938F2DE0918F2DF0910C
:1030E000902D80818032A1F30895E0918F2DF09191
:1030F000902D808190E0C0970A97E8F019C0CA012E
:10310000B3E0880F991FBA95E1F7440F551F480F98
:10311000591F460F571F3196F093902DE0938F2D36
:103120004217530710F09A010AC081E080937A2D6C
:1031300040E050E010C040E050E020E030E0E0919E
:103140008F2DF091902D8081682F70E0605370403A
:103150006A307105A0F2CA010895E091862DF091C0
:10316000872D81939193F093872DE093862D089579
:10317000E091862DF091872D918380831282339682
:10318000F093872DE093862D089590E006C0319648
:10319000F093902DE0938F2D9F5FE0918F2DF09114
:1031A000902D8081803299F39923C1F0A091862DD2
:1031B000B091872D923058F0FD018FE781931196E1
:1031C0009C933196F093872DE093862D0895FD0111
:1031D0008EE78193F093872DE093862D0895E091FB
:1031E0008F2DF091902D8081089580918F2D909159
:1031F000902D01969093902D80938F2D0895E091BE
:10320000862DF091872D6193719381939193F09323
:10321000872DE093862D0895282FE091862DF0913B
:10322000872D809154069091550680589F4FE8173E
:10323000F90721F484E180937A2D08952083809109
:10324000862D9091872D01969093872D8093862DC2
:103250000895AF92BF92CF92DF92FF920F931F9388
:10326000CF93DF935C016B01C0E0D0E013C0F501A8
:10327000EC0FFD1F808190E00E94163F8C018F2D86
:1032800090E00E94163F0817190719F0C0E0D0E03F
:1032900007C02196F601EC0FFD1FF080FF2039F7E3
:1032A000CE01DF91CF911F910F91FF90DF90CF90D2
:1032B000BF90AF9008950F931F93182F092F8091FF
:1032C0008F2D9091902D612F702F0E942919892B9D
:1032D00019F4A0E0B0E013C0E12FF02FDF010D9052
:1032E0000020E9F71197AE1BBF0B80918F2D9091B5
:1032F000902D8A0F9B1F9093902D80938F2DCD0141
:103300001F910F91089515C11092B9050E94C5181B
:103310008CE091E00E945B19892B19F00E94161C29
:10332000F2C081E191E00E945B19892B19F00E94A3
:10333000091EE9C085E191E00E945B19892B19F013
:103340000E94F822E0C08AE191E00E945B19892B7B
:1033500019F00E944E21D7C082E291E00E945B19D1
:10336000892B19F00E94361ECEC088E291E00E949F
:103370005B19892B19F00E94321EC5C08DE291E0C5
:103380000E945B19892B19F00E945924BCC080E36C
:1033900091E00E945B19892B19F00E94AE1BB3C00B
:1033A00087E391E00E945B19892B19F00E94C323E7
:1033B000AAC08AE391E00E945B19892B19F00E9450
:1033C0001923A1C080E491E00E945B19892B19F0B8
:1033D0000E94AB2298C086E491E00E945B19892B81
:1033E00019F00E9453238FC08AE491E00E945B1978
:1033F000892B19F00E94052386C08FE491E00E947A
:103400005B19892B19F00E94B91B7DC084E591E0FE
:103410000E945B19892B19F00E94592174C08AE51A
:1034200091E00E945B19892B19F00E94C41B6BC0AC
:103430008EE591E00E945B19892B19F00E941E1CF9
:1034400062C082E691E00E945B19892B19F00E940C
:10345000E62259C086E691E00E945B19892B19F09B
:103460000E94CF1B50C08BE691E00E945B19892B14
:1034700019F00E94DA1B47C081E791E00E945B19B6
:10348000892B19F00E9447223EC087E791E00E94F5
:103490005B19892B19F00E94C82535C08DE791E092
:1034A0000E945B19892B19F00E94C4252CC083E867
:1034B00091E00E945B19892B19F00E94CC2523C052
:1034C00087E891E00E945B19892B19F00E94AF22D6
:1034D0001AC08EE891E00E945B19892B19F00E94B6
:1034E000A72211C080E991E00E945B19892B19F095
:1034F0000E941A1C08C082E991E00E945B19892B86
:1035000091F50E94051E80917A2D882361F50E9415
:10351000C518E0918F2DF091902DE081EA3319F4D8
:103520000E949A1B06C0ED3021F082E080937A2D34
:103530000895E0918F2DF091902D80818D3009F0CC
:10354000E3CEE091862DF091872D8DE780838091E9
:10355000BE05882341F42091862D8CEA93E3281B35
:103560002F5F2093AE3308951F93182F90E00E9491
:10357000FC3E892B39F420E030E0812F90E0C097A9
:103580000A9710F421E030E0C9011F9108950F93CC
:103590001F9304E91DE2C8010E94BE0DF8010190CD
:1035A0000020E9F731978DE080831093902D0093F0
:1035B0008F2D1F910F910895DF92EF92FF920F933D
:1035C0001F93DF93CF9300D0CDB7DEB70E942413B3
:1035D0000E94532D0E943E2D87EB95E0BE016F5F48
:1035E0007F4F0E940C0D8091B7059091B8052981FD
:1035F0003A81820F931F90939F3380939E330E9452
:10360000AF12892B11F00E941C290E94340D0E94D8
:10361000340D0E948D0D81E097E10E947F0D81ECB9
:1036200096E10E947F0D81E08093BE051CEAE12EA9
:1036300013E3F12EDD24D3948091BE05882321F07D
:1036400085E197E10E947F0D1092BE0510927A2DC0
:1036500010924E060E94340D8EE30E949E0D0E9431
:10366000C71A05C03196F093902DE0938F2DE0910D
:103670008F2DF091902D80818032A1F384E19EE224
:1036800069E975E04EE10E94F41788E19EE26BE77C
:1036900074E04CE30E94EE170E94202C892B61F607
:1036A0000091A2331091A333F092872DE092862DE2
:1036B000109298050E9475189C010097D1F0E09136
:1036C0008F2DF091902D80818D3021F4C9010E94C1
:1036D0009A2D24C01092BE05E091862DF091872D81
:1036E0003183208312823396F093872DE093862DC9
:1036F00002C0D092BE0580917A2D882379F40E9471
:10370000831980917A2D882349F48091BE058823FE
:1037100019F00E94D72602C00E947E2E80917A2D39
:10372000882309F489CF0E94E9211093A3330093E1
:10373000A23382CFE091862DF091872D8AE7819385
:10374000F093872DE093862D80918F2D9091902D71
:1037500001969093902D80938F2D0895E091862D62
:10376000F091872D84E18193F093872DE093862D4E
:103770000895E091862DF091872D87E18193F09354
:10378000872DE093862D0895E091862DF091872D69
:1037900088E18193F093872DE093862D0895E09141
:1037A000862DF091872D86E08193F093872DE0930D
:1037B000862D0895E091862DF091872D87E08193E5
:1037C000F093872DE093862D0895A091862DB091DA
:1037D000872DFD01819311961C9211973196F093DC
:1037E000872DE093862D22E0E0918F2DF091902D92
:1037F0008191F093902DE0938F2DE091862DF091A3
:10380000872D8193F093872DE093862D8D3011F0D5
:103810002F5FEACF80918F2D9091902D01979093FB
:10382000902D80938F2D11962C9308958CE00E94FB
:10383000E51B089584E40E94E51B08958AE00E9438
:10384000E51B089587E991E00E945B19892B11F02F
:1038500082E308958AE991E00E945B19892B11F0B7
:1038600083E308958DE991E00E945B19892B11F0A3
:1038700085E3089580EA91E00E945B19892B11F09D
:1038800080E3089582EA91E00E945B19892B11F090
:1038900081E3089584EA91E00E945B19892B11F479
:1038A00080E0089584E3089586EA91E00E945B1920
:1038B000892B11F080E208958AEA91E00E945B1959
:1038C000892B11F081E208958DEA91E00E945B1945
:1038D000892B11F480E0089582E2089581EB91E054
:1038E0000E945B19892B11F080E4089583EB91E02D
:1038F0000E945B19892B11F081E4089585EB91E01A
:103900000E945B19892B11F080E5089587EB91E007
:103910000E945B19892B11F081E5089589EB91E0F4
:103920000E945B19892B11F082E508958DEB91E0DF
:103930000E945B19892B11F480E0089580E60895B8
:103940009F92AF92BF92CF92DF92EF92FF920F932E
:103950001F93182F00E061E7962E50E7B52E43E73E
:10396000A42E34E7D32E22E7C22E90E1E92E81E186
:10397000F82E0E94C51883EB91E00E945B19892BF9
:1039800031F0E091862DF091872DC1922FC08FEB01
:1039900091E00E945B19892B31F0E091862DF09126
:1039A000872DD19223C083EC91E00E945B19892B73
:1039B00031F0E091862DF091872DA19217C087EC10
:1039C00091E00E945B19892B31F0E091862DF091F6
:1039D000872DB1920BC089EC91E00E945B19892B75
:1039E00049F0E091862DF091872D9192F093872DEB
:1039F000E093862D0E94C518E0918F2DF091902DB7
:103A000080818832B9F5E091862DF091872DE19281
:103A1000F093872DE093862D80918F2D9091902D9E
:103A200001969093902D80938F2D812F0E94A01C42
:103A300080917A2D882309F077C0E0918F2DF09145
:103A4000902D8081893211F084E060C0E091862D54
:103A5000F091872DF192F093872DE093862D809140
:103A60008F2D9091902D01969093902D80938F2D76
:103A700011E01EC00E94A61F982F882369F40E949F
:103A8000D025982F882341F40E949D0F982F8823DA
:103A900019F40E948420982F80917A2D882309F0B0
:103AA00043C0112321F0911711F085E02FC0192F89
:103AB0000E94C518E0918F2DF091902DE081ED309E
:103AC00099F1EA3389F1EC3279F1EB3369F1E932BA
:103AD00059F11130C1F40E946E1C8823D9F40E9460
:103AE000541C8823B9F48091B905882339F0002348
:103AF000D9F40E94221C882361F407C080914D34C0
:103B0000882319F011C083E101C086E080937A2DEB
:103B10000BC001E0E091862DF091872D8193F09309
:103B2000872DE093862D25CF1F910F91FF90EF9069
:103B3000DF90CF90BF90AF909F9008951F930E9409
:103B40009D0F182F882329F40E948420182F882382
:103B500011F180917A2D8823F1F40E94C518E0912B
:103B60008F2DF091902D8191F093902DE0938F2DDA
:103B70008D3321F083E080937A2D0DC0E091862D66
:103B8000F091872D89E78193F093872DE093862D1F
:103B9000812F0E94A01C1F910895E091862DF09125
:103BA000872D8193F093872DE093862D0E94C51871
:103BB00083EC91E00E945B19892B31F0E091862D16
:103BC000F091872D83E717C08FEB91E00E945B197E
:103BD000892B31F0E091862DF091872D84E70BC081
:103BE00087EC91E00E945B19892B51F0E091862DC2
:103BF000F091872D80E78193F093872DE093862DB8
:103C00000E94C5180E949E1D089582E00E94CD1D4D
:103C1000089581E00E94CD1D0895E091862DF091D8
:103C2000872D8193F093872DE093862D0E94C518F0
:103C3000E091862DF091872D88EA8193F093872D6E
:103C4000E093862D0E9475189C01009719F482E17B
:103C500080937A2D80917A2D882319F4C9010E94CE
:103C6000AD18089582E10E940D1E08958FE00E9414
:103C70000D1E0895E0918F2DF091902D8081883256
:103C800019F424E930E002C020E030E0C9010895D1
:103C9000282FDB014091A2335091A333FA01819385
:103CA000F093A333E093A23390E08C91E091A233A0
:103CB000F091A3338193F093A333E093A2338C91DB
:103CC000811111969F5F9E3081F7243851F024397D
:103CD00041F0223811F494E005C0213811F088E059
:103CE0001BC095E081E02091A2333091A333F9010C
:103CF0001192F093A333E093A2338F5F981798F754
:103D00003093A3332093A23380917F2D9091802D07
:103D10008217930730F489E080937A2DEFEFFFEF5D
:103D200007C08091BF059091C005FA01E81BF90B0F
:103D3000CF0108950F931F93CF93DF93E0918F2DC1
:103D4000F091902D808190E0C0970A9728F420E0B0
:103D500030E040E050E025C082E016C0CA01B90161
:103D60002AE030E040E050E00E947E3E9B01AC0142
:103D7000CE01AA2797FDA095BA2F280F391F4A1FF9
:103D80005B1F57FF08C08AE080937A2D20E030E067
:103D900040E050E012C00F5F1F4F1093902D009332
:103DA0008F2D00918F2D1091902DF8018081C82FBB
:103DB000D0E0E097CA30D10588F2B901CA01DF919D
:103DC000CF911F910F910895CF93DF93C091862DCE
:103DD000D091872DDE0182EA8D93CD0101969093DB
:103DE000872D8093862DE0918F2DF091902D21913C
:103DF00011962C9301969093872D8093862DF093A6
:103E0000902DE0938F2D22E018C08D3019F480930F
:103E10007A2D2DC0E091862DF091872D8193F0931E
:103E2000872DE093862D80918F2D9091902D019676
:103E30009093902D80938F2D2F5FE0918F2DF09197
:103E4000902D8081823209F7E091862DF091872DA7
:103E50008193F093872DE093862D80918F2D909103
:103E6000902D01969093902D80938F2D2983DF9133
:103E7000CF91089590E00E94033F0895BF92CF92A2
:103E8000DF92EF92FF920F931F93CF93DF93E09116
:103E90008F2DF091902D808190E00E94033F892B1F
:103EA00029F0EE24FF248701BB2433C08BE023C01C
:103EB0009E0120533040D801C70144E0880F991F6C
:103EC000AA1FBB1F4A95D1F72A30310530F479017A
:103ED0000027F7FC0095102F06C0E7977E0100270A
:103EE000F7FC0095102FE80EF91E0A1F1B1F89E032
:103EF000B81639F48CE080937A2DEE24FF248701E4
:103F000019C0B3940894C11CD11CD092902DC092BA
:103F10008F2DC0908F2DD090902DF601808190E054
:103F20000E94163FC82FD0E0CE010E94033F892B8C
:103F300009F0BECFB701C801DF91CF911F910F915A
:103F4000FF90EF90DF90CF90BF9008950F931F9355
:103F5000DF93CF9300D000D0CDB7DEB700918F2D87
:103F60001091902DF8018081823229F40E94E41E84
:103F700022E030E04FC0843259F40F5F1F4F10939E
:103F8000902D00938F2D015010400E943E1F0EC0B7
:103F900090E00E94FC3E892B39F0CE0101960E94F0
:103FA0008417882339F434C00E949A1E69837A8367
:103FB0008B839C8380917A2D882351F5E091862D07
:103FC000F091872D84EA8193F093872DE093862DDD
:103FD00069817A818B819C810E94FF1880918F2D4D
:103FE000801B03C0F80181918F01E091862DF09133
:103FF000872D8193F093872DE093862D80918F2DCF
:104000009091902D0817190768F321E030E002C065
:1040100020E030E0C9010F900F900F900F90CF91EA
:10402000DF911F910F910895CF93DF93EC01E88109
:10403000F9818081843981F47396F983E8837397D9
:1040400087859089009701F1DC012D913D91220F28
:10405000331F220F331F10C0843841F4DF011F9635
:104060007396F983E88324E030E006C088E080930B
:104070007A2D0E94E92108C080E090E002C01D92E4
:10408000019682179307D8F3DF91CF910895EF92AD
:10409000FF920F931F93CF93DF93E82E8B01FB01C9
:1040A00001900020E9F73197FE2EF61AC091BF0566
:1040B000D091C0051CC08E1581F4BE016F5F7F4F8B
:1040C000C8010E942919F81641F48091BF0590910A
:1040D000C005BE01681B790B0FC08881843831F0A0
:1040E000843921F088E080937A2D04C0639688811A
:1040F000882309F76FEF7FEFCB01DF91CF911F91FD
:104100000F91FF90EF9008951F93CF93DF93E7E611
:10411000F4E0119284E0E637F807D9F7C0918F2DCB
:10412000D091902D1881812F90E00E94FC3E892B28
:1041300041F0109367042196D093902DC0938F2D5A
:1041400003C087E080937A2DC8E6D4E0E0918F2DFC
:10415000F091902D80810E94B41A892B71F0E0912A
:104160008F2DF091902D81918993F093902DE09374
:104170008F2D84E0C537D80749F7E0918F2DF09156
:10418000902D8081883219F484E990E002C080E0AB
:1041900090E080937604882321F484E88093760469
:1041A00005C03196F093902DE0938F2D80917A2D5C
:1041B000882309F051C08091760467E674E00E947C
:1041C00047209C0180917A2D882309F045C08FEF0C
:1041D0002F3F3807C1F490917604943931F48091DF
:1041E0009805882311F488E135C0892F67E674E0CB
:1041F0000E94481E9C018FEF2F3F380769F1809184
:104200007A2D882349F580917604E091862DF091EE
:10421000872D8193F093872DE093862DC9010E940D
:10422000AD1880917604843949F5E091862DF0919E
:10423000872D80E18193F093872DE093862D81E097
:104240000E94A01CE0918F2DF091902D80818932E9
:1042500031F08EE080937A2D20E030E01AC0319664
:10426000F093902DE0938F2DE091862DF091872D86
:1042700081E18193F093872DE093862D80917604E0
:10428000843829F0843919F022E030E002C021E0BE
:1042900030E0C901DF91CF911F910895E091862D03
:1042A000F091872D8EE08193F093872DE093862DFA
:1042B0000895E091862DF091872D8AE18193F09306
:1042C000872DE093862D0895E091862DF091872D1E
:1042D0008CE08193F093872DE093862D08958F9243
:1042E0009F92AF92BF92CF92DF92EF92FF920F9385
:1042F0001F93DF93CF93CDB7DEB764970FB6F894D3
:10430000DEBF0FBECDBF7B018C011C8A97FF11C0A1
:104310008DE20E949E0DAA24BB246501AE18BF0841
:10432000C00AD10A82E1F82E4E010894811C911C2A
:1043300026C0611571058105910519F05B016C01BD
:10434000F1CF80E30E949E0D28C0080D191DC60103
:10435000B5012AE030E040E050E00E94BD3E605DE3
:10436000F8016083FA94C601B5012AE030E040E02C
:1043700050E00E94BD3EC901DA015C016D010F2DC4
:1043800010E0A114B104C104D104F9F60F5F1F4F6E
:10439000C401800F911F0E94920D64960FB6F8948D
:1043A000DEBF0FBECDBFCF91DF911F910F91FF9068
:1043B000EF90DF90CF90BF90AF909F908F90089537
:1043C00098E2899FC00111248C599F4F0E947F0D54
:1043D0000895CF93DF9380914E068823D1F089E32F
:1043E00097E10E947F0D60917A2D70E080E090E06F
:1043F0000E946F218FE297E10E947F0D6091912DC5
:104400007091922D80E090E00E946F218CE297E104
:1044100032C00E94340D0E94340DC4E9DDE202C0B6
:104420000E949E0D89918D30D9F70E94340D24E9A8
:104430003DE204C08AE20E949E0D9E01E9012196A0
:1044400080918F2D9091902D02972817390790F326
:1044500088E297E10E947F0D0E94340D80E297E18F
:104460000E947F0D60917A2D70E080E090E00E94C4
:104470006F218DE197E10E947F0D80917A2D0E943E
:10448000E02181E08093772DDF91CF910895809195
:10449000B9058F5F8093B905E091862DF091872D46
:1044A00089E18193F093872DE093862D80E00E942F
:1044B000A01C08950F931F93E091862DF091872DF6
:1044C0008193F093872DE093862D0E94C5180BE70A
:1044D0001CE731C080E00E94A01C80917A2D8823C7
:1044E00099F50E94C518E0918F2DF091902DE081F3
:1044F000EC3231F4E091862DF091872D108307C0C6
:10450000EB3311F5E091862DF091872D008380919A
:104510008F2D9091902D01969093902D80938F2DBB
:104520008091862D9091872D01969093872D809371
:10453000862D0E94C518E0918F2DF091902DE0817D
:10454000ED3011F0EA3331F61F910F91089583E4B5
:104550000E945A22089583E00E945A220895E09111
:10456000862DF091872D83E28193F093872DE09340
:10457000862D0E94C5180E94842008951F931CE771
:104580000E94C5180E94842080917A2D8823E1F42E
:104590000E94C518E0918F2DF091902D80818C3272
:1045A00099F4E091862DF091872D1193F093872D4A
:1045B000E093862D80918F2D9091902D0196909370
:1045C000902D80938F2DDCCF1F91089581E08093F3
:1045D0009805E091862DF091872D89E08193F093E5
:1045E000872DE093862D0E94BE2210929805089593
:1045F000E091862DF091872D8DE08193F093872DAA
:10460000E093862D0E94BE220895E091862DF091C0
:10461000872D85E08193F093872DE093862D0E946E
:10462000C5180E948420019719F082E080937A2DAA
:104630000895E091862DF091872D86E18193F09386
:10464000872DE093862D0E94C518E0918F2DF09163
:10465000902D8081823221F50E94E41E80917A2D76
:10466000882301F5E0918F2DF091902D80818C327F
:1046700021F082E080937A2D0895E091862DF091CB
:10468000872D8CE78193F093872DE093862D809181
:104690008F2D9091902D01969093902D80938F2D3A
:1046A0000E94BE2208951F9381E080934D34E091D3
:1046B000862DF091872D84E08193F093872DE093F0
:1046C000862D0E94C5180E948420182F0E94C518AC
:1046D000113059F4E0918F2DF091902D8191F0934C
:1046E000902DE0938F2D8D3311F083E02EC0E0915B
:1046F000862DF091872D89E78193F093872DE093A4
:10470000862D81E00E94A01C80917A2D8823C9F516
:104710000E94C5188DEC91E00E945B19892BA1F0D5
:10472000E091862DF091872D87E38193F093872D7B
:10473000E093862D0E94C51881E00E94A01C809104
:104740007A2D8823F1F404C081E180937A2D19C079
:104750000E94C51880ED91E00E945B19892B79F0C9
:10476000E091862DF091872D8AE38193F093872D38
:10477000E093862D0E94C51881E00E94A01C109233
:104780004D341F910895E091862DF091872D85E19C
:104790008193F093872DE093862D0E94C518809118
:1047A000B9058F5F8093B90581E00E94A01C8091BC
:1047B0007A2D882309F07CC00E94C51885ED91E010
:1047C0000E945B19892BB9F1E091862DF091872D1C
:1047D00088E38193F093872DE093862D0E94C5187E
:1047E000E0918F2DF091902D808190E0C0970A97F5
:1047F000D8F4E091862DF091872D88EA8193F0938B
:10480000872DE093862D0E9475189C01009719F45E
:1048100082E180937A2D80917A2D882309F048C017
:10482000C9010E94AD180BC00E94831980917A2D96
:10483000882329F0089580E180937A2D08950E94BD
:10484000C5188AED91E00E945B19892B89F1E091EE
:10485000862DF091872D89E38193F093872DE09346
:10486000862D0E94C518E0918F2DF091902D8081AA
:1048700090E0C0970A97D0F4E091862DF091872DB3
:1048800088EA8193F093872DE093862D0E94751816
:104890009C01009719F482E180937A2D80917A2D02
:1048A000882331F4C9010E94AD1808950E9483192C
:1048B0000895FF920F931F93E091862DF091872D1D
:1048C00083E18193F093872DE093862D0E94C51894
:1048D00081E00E94A01C80917A2D882309F056C0A7
:1048E0000E94C5188FED91E00E945B19892B19F089
:1048F0000E94321E0CC084EE91E00E945B19892B4D
:1049000019F00E94361E03C08FE080937A2D8091AB
:104910007A2D8823D9F50E94C5189CE7F92E08EA5C
:1049200012E12DC0E091862DF091872DF192F09348
:10493000872DE093862D80918F2D9091902D01965B
:104940009093902D80938F2D0E94C518E091862D15
:10495000F091872D0193F093872DE093862D0E948F
:1049600075189C01009711F410937A2D80917A2D7F
:10497000882361F4C9010E94B8180E94C518E0910B
:104980008F2DF091902D80818C3261F21F910F91CB
:10499000FF900895DF92EF92FF920F931F93CF93B2
:1049A000DF938B017A01C091862DD091872DDE0196
:1049B0008D93B093872DA093862DE0918F2DF0914C
:1049C000902D8081883239F580E189831196B093EA
:1049D000872DA093862D80918F2D9091902D0196FB
:1049E0009093902D80938F2D8CE7D82EF701819195
:1049F0007F010E94A01C80917A2D8823D9F5015057
:104A00001040E0918F2DF091902D01151105C1F00E
:104A100080818C3211F082E017C0E091862DF091F8
:104A2000872DD192F093872DE093862D80918F2D45
:104A30009091902D01969093902D80938F2DD6CFAD
:104A40008081893221F08EE080937A2D13C0E0912D
:104A5000862DF091872D81E18193F093872DE0934E
:104A6000862D80918F2D9091902D01969093902D71
:104A700080938F2DDF91CF911F910F91FF90EF9039
:104A8000DF900895DF93CF930F92CDB7DEB791E01B
:104A9000998361E070E0AE014F5F5F4F0E94CA24CE
:104AA00081E00F90CF91DF91089583E10E9442252C
:104AB000089582E10E94422508958AE00E944225DD
:104AC000089580E10E94422508958FE00E944225CA
:104AD000089589E00E94422508958EE00E944225B3
:104AE00008958DE00E94422508958BE00E944225A2
:104AF00008958CE00E944225089583E00E9442259B
:104B000090E0089581E10E94422508958BE00E9483
:104B10004225089587E00E94422590E0089586E0AE
:104B20000E94422590E0089585E00E94422590E091
:104B3000089584E00E94422590E0089582E00E945A
:104B4000422590E008950E9442250E94C518E091F8
:104B50008F2DF091902D8191F093902DE0938F2DDA
:104B60008D3321F083E080937A2D0895E091862D96
:104B7000F091872D89E78193F093872DE093862D1F
:104B800081E00E94A01C08958DE10E94A325089554
:104B90008CE10E94A32508958BE10E94A32508952E
:104BA000CF93DF93C091862DD091872D86E38883A4
:104BB0008091862D9091872D01969093872D8093DB
:104BC000862D8AEE91E00E945B19892B19F00E94D4
:104BD0009E2595C08FEE91E00E945B19892B19F0FC
:104BE0000E9499258CC083EF91E00E945B19892B6C
:104BF00019F00E947D2583C088EF91E00E945B1927
:104C0000892B19F00E9494257AC08CEF91E00E94C4
:104C10005B19892B19F00E948F2571C080E092E00A
:104C20000E945B19892B19F00E948A2568C084E0D4
:104C300092E00E945B19892B19F00E946D255FC0DC
:104C400089E092E00E945B19892B19F00E9471257E
:104C500056C08EE092E00E945B19892B19F00E94E9
:104C600075254DC082E192E00E945B19892B19F0F5
:104C70000E94652544C089E192E00E945B19892B5E
:104C800019F00E9461253BC080E292E00E945B190E
:104C9000892B19F00E94692532C085E292E00E94BA
:104CA0005B19892B19F00E94822529C08AE292E0C3
:104CB0000E945B19892B19F00E94592520C080E3BE
:104CC00092E00E945B19892B19F00E94552517C0AC
:104CD00086E392E00E945B19892B19F00E945D2502
:104CE0000EC08AE392E00E945B19892B19F00E94A2
:104CF000792505C0D093872DC093862D80E0DF9164
:104D0000CF9108951F93CF93DF93DB01EC018A814C
:104D10006AE00E949D3E805DFD0181938A810E9430
:104D20009D3E905D11969C93DF0111961AE31183CD
:104D3000AD014F5F5F4F89810E949D3E805D11965E
:104D40008C93FA01319689810E949D3E905DDA0133
:104D500011969C93DF0111961183FD013196888194
:104D60000E949D3E805D11968C9388810E949D3E9D
:104D7000905D91831282DF91CF911F9108950895E4
:104D80000895E091862DF091872D80818E3719F05E
:104D90008F3761F406C03196F093872DE093862D0E
:104DA00008953296F093872DE093862D08958CEA2E
:104DB00093E39093872D8093862D0E94C1261DC07A
:104DC0000E94C126E091862DF091872D8191F0936C
:104DD000872DE093862D90E001979C01220F331FD1
:104DE000280F391F220F331F220F331F2452354F34
:104DF000F90185919491FC010995E091862DF0913E
:104E0000872D80818D3721F080917A2D8823C1F202
:104E100008958AE08093A8338091852D882371F0CE
:104E20001092852D89E380937A2D8091760590915B
:104E300077059093AB338093AA3381E008950F9365
:104E40001F93DF93CF9300D0CDB7DEB70E943E2DE6
:104E50008091BF059091C0059A8389838E010F5F71
:104E60001F4F03C0C8010E941420E981FA8180818C
:104E70008823C1F70F900F90CF91DF911F910F9171
:104E800008950E941F271092852D1092A9338AE061
:104E90008093A8331092772D10925F0610925E06D1
:104EA0000895DF93CF93CDB7DEB764970FB6F8942C
:104EB000DEBF0FBECDBF20918A2D30918B2D80910A
:104EC0007205909173052817390791F08BE697E1E9
:104ED0000E947F0DCE0101960E94BE0D8981893707
:104EE00011F0893549F40E94532D89E597E102C0FC
:104EF00081E497E10E947F0D64960FB6F894DEBFBF
:104F00000FBECDBFCF91DF91089507C03196F093CA
:104F10007804E09377040E949E0DE0917704F0916D
:104F2000780480818D3791F708950F931F93CF9365
:104F3000DF93A0917704B0917804FD012191F09363
:104F40007804E09377042633F1F1273330F42A30E4
:104F500021F12C3009F04DC026C02E37D1F02F376B
:104F600021F0243409F045C01BC011968C91319674
:104F7000F0937804E0937704C0E0D0E0082F10E0CD
:104F800004C080E20E949E0D2196C017D107CCF389
:104F900040C080E20E949E0D3CC088EC97E105C0B5
:104FA00086EC97E102C081EC97E10E947F0D809131
:104FB0007704909178040196909378048093770415
:104FC0000E94852726C011962C913196F093780483
:104FD000E093770430E021503040C901880F991FD9
:104FE000820F931F880F991F880F991F8251964F28
:104FF0000EC030E021503040C901880F991F820F48
:10500000931F880F991F880F991F8252954F0E94F6
:105010007F0DDF91CF911F910F9108951F9390E025
:105020000196E0917704F0917804E80FF91FF0936E
:105030007804E09377041191F0937804E093770477
:105040000CC0E0917704F09178048191F09378049A
:10505000E09377040E949E0D1150112391F71F9148
:10506000089580E00E940E28089584E00E940E2892
:10507000089584E00E940E2808950F931F93CF9304
:10508000DF93E0917704F0917804818192813396E7
:10509000F0937804E0937704C091BF05D091C005E8
:1050A000C80FD91F8E01025F1F4F8981882311F01D
:1050B0000E949E0D2196C017D107B9F7DF91CF91BD
:1050C0001F910F9108950E943D280895E091862D2B
:1050D000F091872D82819F01280F311D3093770534
:1050E00020937605819191919093922D8093912DAB
:1050F000F093872DE093862D80916B05882389F0AE
:105100008BE50E949E0D6091912D7091922D80E013
:1051100090E00E946F218DE50E949E0D80E20E942A
:105120009E0D0895E0917704F09178046181728179
:105130003396F0937804E0937704882777FD809581
:10514000982F0E946F2108955CC00E94662880916C
:10515000862D9091872D01969093872D8093862D93
:105160003AC00E94C126E091862DF091872D819151
:10517000F093872DE093862D8F3041F40E94FD3609
:1051800080917A2D882309F041C082E190E0019757
:105190009C01220F331F280F391F220F331F220FAC
:1051A000331F2452354FF90185919491FC010995E3
:1051B00080917A2D882351F58091A833882319F0A6
:1051C00081508093A8338091A833882321F40E94D2
:1051D00009278823D9F4E091862DF091872D8081CD
:1051E0008D3709F0BECF9F012F5F3F4F8091720531
:1051F000909173052817390749F03093872D209334
:10520000862D80917A2D882309F49FCF089580916F
:10521000772D882359F48091AA339091AB339093E2
:10522000872D8093862D0E94A428089585E280937F
:105230007A2D0E94E92108950E94340D0E94412791
:1052400081E080934E0620918A2D30918B2D8091A4
:105250007205909173052817390729F482EA97E1BE
:105260000E947F0D08953093872D2093862D3093D3
:105270007705209376050E94A42880917A2D8823B3
:1052800011F00E94E9210E94340D08950F931F939D
:10529000DF93CF93CDB7DEB72F970FB6F894DEBF6D
:1052A0000FBECDBFE0917704F091780481819281A7
:1052B0003396F0937804E09377048E010F5F1F4FCD
:1052C000B8010E948B0FC8010E94920D2F960FB655
:1052D000F894DEBF0FBECDBFCF91DF911F910F912C
:1052E0000895E0917704F0917804E081E93870F452
:1052F000E13821F0E238D9F1E43819F40E943D2870
:105300000895E33869F50E9446290895E93A60F561
:10531000E13A19F40E9439280895E23A19F40E94FA
:1053200031280895E83A19F40E9492280895E43A41
:1053300019F40E9435280895E43991F40E943D281B
:1053400007C0E7FF03C00E94712902C00E94952791
:10535000E0917704F0917804E081ED3791F70895BA
:1053600088E080937A2D089588E080937A2D0895BF
:105370006F927F928F929F92AF92BF92CF92DF9265
:10538000EF92FF920F931F93DF93CF93CDB7DEB7CA
:10539000CF58D0400FB6F894DEBF0FBECDBF0E94ED
:1053A0006718E0918F2DF091902D1081812F90E062
:1053B0000E94FC3E892B09F43EC180E492E00E94E9
:1053C0005B19892B09F43EC00E94340D86E492E0FB
:1053D0000E94920DEE24FF248E010F5F1F4FC70124
:1053E00065E070E00E94A93E892B11F40E94340D03
:1053F000C701B8010E948B0F8981882301F1F80150
:1054000001900020E9F73197E01BF10B3E9738F04F
:105410001F860EC0C80167E572E00E942E3FF801AA
:1054200001900020E9F73197E01BF10B3E9790F3D4
:10543000C8010E94920D0894E11CF11CD0CF0E947B
:10544000340DF6C089E592E00E945B19892B09F4BE
:1054500071C00E94340D1091BF050091C0058EE50A
:1054600092E00E94920D812F902F6C01760108949A
:10547000E11CF11CAA24BB2490E1892E912C54C07C
:10548000C50183709070892B11F40E94340DF601D0
:1054900080818438D1F4C7010E94920DF7010190F8
:1054A0000020E9F73197EE19FF0984010E1B1F0B4D
:1054B00006C087E592E00E94920D01501040011550
:1054C0001105B9F783E792E024C0843909F0B0C030
:1054D000C7010E94920D88E792E00E94920D8AE730
:1054E00092E00E94920DF70101900020E9F73197B8
:1054F000EE19FF0984010E1B1F0B06C087E592E021
:105500000E94920D0150104001151105B9F78CE76A
:1055100092E00E94920D0894A11CB11C83E190E0DE
:10552000C80ED91EE80EF91EF6018081882309F005
:10553000A7CF7EC08FE792E00E945B19892B09F408
:1055400073C0A0907704B0907804EE24FF24870104
:1055500080E1882E912C8C0E9D1EB2E16B2E712C59
:105560006C0E7D1E80EF97E10E947F0DC801B70190
:105570000E946F218DEE97E10E947F0D8E2D0E947B
:10558000A50EAB01BC014115510561057105A9F1DD
:10559000C40120E830E00E94BF0EF401C080D18039
:1055A0007092780460927704FFEFCF16FFEFDF066A
:1055B00019F480EE97E123C080E20E949E0DB601AF
:1055C00080E090E00E946F218091770490917804B0
:1055D0000196909378048093770407C0E7FF03C097
:1055E0000E94712902C00E949527E0917704F091F2
:1055F0007804E081ED3791F704C08CEC97E10E94CC
:105600007F0D0E94340D0894E11CF11C011D111D39
:1056100083E0E816F1040105110509F0A3CFB0926B
:105620007804A092770404C085E892E00E94920D6D
:105630000E94340DACC0812F90E0C097E0918A2D7C
:10564000F0918B2D20917205309173050A97A0F58A
:10565000E217F30709F49BC00E9475189093650642
:10566000809364060E946718E0918F2DF091902D31
:1056700080818D32C1F43196F093902DE0938F2D7F
:105680000E946718E0918F2DF091902D808190E01D
:10569000C0970A9718F40E94751809C08091A43326
:1056A0009091A53304C08091640690916506909313
:1056B000500680934F0612C0E217F30709F467C043
:1056C0008091A4339091A5339093500680934F0618
:1056D0008081918190936506809364062091640691
:1056E0003091650680914F0690915006821793077E
:1056F00008F44DC0C9010E946F2D909378048093E7
:1057000077040E94340DE0917704F0917804809141
:10571000720590917305E817F907C8F50191119189
:10572000F0937804E093770480914F0690915006AF
:105730008017910760F180E20E949E0DB80180E021
:1057400090E00E946F2180917704909178040196F7
:10575000909378048093770407C0E7FF03C00E940A
:10576000712902C00E949527E0917704F091780496
:10577000E081ED3791F70E94340D8091770490918C
:10578000780401969093780480937704BCCFC15736
:10579000DF4F0FB6F894DEBF0FBECDBFCF91DF91C4
:1057A0001F910F91FF90EF90DF90CF90BF90AF903F
:1057B0009F908F907F906F900895DF92EF92FF926D
:1057C0000F931F937C018B01DC0113968C9113972F
:1057D0006AE00E949D3E805DF801819313968C9152
:1057E0000E949D3E905DD80111969C9320E2D22E9E
:1057F000D182CF0102966BEC72E00E94393FF80132
:10580000D682D70115968C91159764E60E949D3E2D
:10581000892F6AE00E949D3E805D878315968C915A
:1058200064E60E949D3E892F6AE00E949D3E905D45
:10583000908711861F910F91FF90EF90DF90089550
:105840008FEC92E00E945B19892B19F00E94B82915
:105850004AC084ED92E00E945B19892B19F00E94E6
:105860001C2941C088ED92E00E945B19892B19F038
:105870000E94512738C08CED92E00E945B19892B61
:1058800019F00E9407292FC081EE92E00E945B1957
:10589000892B19F00E941F2726C087EE92E00E94F4
:1058A0005B19892B19F00E947A2C1DC08CEE92E0B6
:1058B0000E945B19892B19F00E94631214C081EFBA
:1058C00092E00E945B19892B19F00E94E4140BC02E
:1058D00086EF92E00E945B19892B19F420E030E0FA
:1058E00004C00E94CB2C21E030E0C9010895089546
:1058F000089508950E94340D88E498E10E947F0D78
:105900006091782D7091792D2091720530917305F9
:10591000621B730B882777FD8095982F0E946F215B
:105920008CE398E10E947F0D0E94340D8AE298E199
:105930000E947F0D60917F2D7091802D2091A23368
:105940003091A333621B730B882777FD8095982FC6
:105950000E946F218EE198E10E947F0D0E94340D1C
:105960008FEF97E10E947F0D60919E3370919F337E
:105970002091B7053091B805621B730B882777FD1E
:105980008095982F0E946F2183EF97E10E947F0DF1
:105990000E94340D08951F930E946718E0918F2D87
:1059A000F091902D80818D3081F50E94AA12182FE0
:1059B0008D3528F48A3558F48535C9F405C08F3FF4
:1059C000B1F48CED98E152C085EC98E14FC08FEABC
:1059D00098E10E947F0D1A3511F480E305C01B3554
:1059E00011F481E301C082E30E949E0D0AC086E9A2
:1059F00098E10E947F0D612F70E080E090E00E94AE
:105A00006F218EE20E949E0D33C08DEF92E00E94C6
:105A10005B19892B19F08FEF90E023C081E093E0B0
:105A20000E945B19892B19F085E590E01AC084E08B
:105A300093E00E945B19892B19F08AE590E011C070
:105A400088E093E00E945B19892B19F08BE590E0C8
:105A500008C08CE093E00E945B19892B29F08CE54B
:105A600090E00E94CC1604C089E598E10E947F0D69
:105A70001F910895089508950895089588E19EE27C
:105A80006BE774E04CE30E94EE1784E19EE269E963
:105A900075E04EE10E94F41710926C0510925106C9
:105AA00010928E2D08950E94A40C1092A53310928E
:105AB000A4331092BE050895FB01E80FF91FDB0126
:105AC00002C081918D938091720590917305E817C2
:105AD000F907B8F3B0937305A093720508959C017C
:105AE000E0918A2DF0918B2D80819181821793070F
:105AF00014F0CF0108958281E80FF11DF5CFE091F8
:105B00008A2DF0918B2D409172055091730520E004
:105B100030E00BC0208131812115310519F420E0DE
:105B200030E006C08281E80FF11DE417F50791F718
:105B3000C90108959C018091A4339091A5338217E7
:105B40009307A0F1E0918A2DF0918B2DDF014D910B
:105B50005D914217530724F04217530739F507C0E8
:105B60008281E82FF0E03297EA0FFB1FEFCF8C9194
:105B7000DF01A80FB11D02C08D9181938091720544
:105B800090917305A817B907B8F3F0937305E093E4
:105B900072058091A4339091A5334817590731F4C9
:105BA0000E947F2D9093A5338093A4330895A091F4
:105BB0007205B0917305FD01E80FF91F8091782DF2
:105BC0009091792D8E179F0720F489E080937A2D8C
:105BD0000895F0937305E09372056150704004C01E
:105BE0008C91808331971197A617B707C9F708954D
:105BF000DC018091AE33282F30E08CEA93E3909360
:105C0000872D8093862D0CC0E091862DF091872DF5
:105C100081918D93F093872DE093862D2150304014
:105C20002115310589F70895CF93DF93EC01809119
:105C3000AE3390E0BE010E94D72D80917A2D88234B
:105C400019F4CE010E94F82DDF91CF910895409173
:105C50007205509173058091AE339A01280F311D62
:105C60008091782D9091792D8217930780F0CA0149
:105C70000E94F82D2091AE338091720590917305AA
:105C8000820F911D9093730580937205089589E0AA
:105C900080937A2D0895CF93DF93EC018A81282F8A
:105CA00030E08091AE33281B31092115310501F117
:105CB00037FF0CC088279927821B930BBE010E94D7
:105CC000D72D80917A2D8823B1F412C0DE01A20F66
:105CD000B31FFE0102C08D91819380917205909156
:105CE0007305A817B907B8F3F0937305E09372052D
:105CF000CE010E94F82DDF91CF910895CF93DF93CD
:105D000081E08093772D8CEA93E39093872D8093A5
:105D1000862DC091AC33D091AD338091A433909156
:105D2000A5338C179D0738F40E94272ED093A533F6
:105D3000C093A43318C0E0918A2DF0918B2D8081FF
:105D400091818C179D0724F0C817D90749F404C026
:105D50008281E80FF11DF3CFCF010E944B2E03C0CB
:105D6000CF010E94142EDF91CF91089590E001970A
:105D7000FC01EE0FFF1FE80FF91FEE0FFF1FEE0FE4
:105D8000FF1FE452F54F85919491009711F0FC01AB
:105D900009950895EF92FF920F931F93CF93DF938E
:105DA0002091192E81E090E0821B9109880F991FA4
:105DB000880F991FC0911A2ED0911B2EC81BD90B8A
:105DC000288139814A815B81CA01AA27BB27F90151
:105DD0000BB68BBF819190810BBE7C0100E010E07F
:105DE0002E5F3F4F4F4F5F4FCA01AA27BB27F901D4
:105DF0000BB68BBF219130810BBEC901A0E0B0E092
:105E0000DC01992788278E0D9F1DA01FB11F888355
:105E10009983AA83BB83DF91CF911F910F91FF904C
:105E2000EF900895CF93DF932091192E81E090E0B9
:105E3000821B9109880F991F880F991FC0911A2EF4
:105E4000D0911B2EC81BD90B88819981AA81BB8157
:105E50009D0144275527FC010BB62BBF80810BBE4B
:105E600090E0A0E0B0E088839983AA83BB83DF91B0
:105E7000CF910895CF93DF932091192E81E090E088
:105E8000821B9109880F991F880F991FC0911A2EA4
:105E9000D0911B2EC81BD90B88819981AA81BB8107
:105EA0009D0144275527FC010BB62BBF81919081A2
:105EB0000BBEA0E0B0E088839983AA83BB83DF9107
:105EC000CF9108952091192E81E090E0821B9109D5
:105ED000880F991F880F991FE0911A2EF0911B2EA1
:105EE000E81BF90B80819181A281B3818095909507
:105EF000A095B09580839183A283B3830895209168
:105F0000192E81E090E0821B9109880F991F880F5C
:105F1000991FE0911A2EF0911B2EE81BF90B80813E
:105F20009181909581959F4FAA2797FDA095BA2FB3
:105F300080839183A283B383089589E280937A2D2D
:105F400008956F927F928F929F92AF92BF92CF925D
:105F5000DF92EF92FF920F931F93CF93DF9388E12D
:105F60009EE268E30E942718AC01CB01DA015C01D4
:105F70006D012091192E81E090E0821B9109880F1C
:105F8000991F880F991FC0911A2ED0911B2EC81BE4
:105F9000D90B288139814A815B81D7FE04C0EE2468
:105FA000FF24870126C039014A0171E0E72EF12C58
:105FB000012D112D19C0C50181709070892B41F000
:105FC000C801B7019301A4010E947E3E7B018C01B0
:105FD000B301C4019301A4010E947E3E3B014C0128
:105FE000D594C794B794A794A114B104C104D10463
:105FF00011F7E882F9820A831B83DF91CF911F9109
:106000000F91FF90EF90DF90CF90BF90AF909F9057
:106010008F907F906F90089588E19EE268E30E94E0
:1060200027184091192E21E030E0241B3109220F5E
:10603000331F220F331FE0911A2EF0911B2EE21B0B
:10604000F30B20813181428153812617370748079E
:10605000590749F081E090E0A0E0B0E080839183AF
:10606000A283B3830895108211821282138208954D
:1060700088E19EE268E30E9427184091192E21E0F2
:1060800030E0241B3109220F331F220F331FE09110
:106090001A2EF0911B2EE21BF30B208131814281DD
:1060A0005381261737074807590749F481E090E0E4
:1060B000A0E0B0E080839183A283B383089510822F
:1060C000118212821382089588E19EE268E30E94A1
:1060D00027184091192E21E030E0241B3109220FAE
:1060E000331F220F331FE0911A2EF0911B2EE21B5B
:1060F000F30B2081318142815381261737074807EE
:1061000059074CF081E090E0A0E0B0E080839183FB
:10611000A283B3830895108211821282138208959C
:1061200088E19EE268E30E9427184091192E21E041
:1061300030E0241B3109220F331F220F331FE0915F
:106140001A2EF0911B2EE21BF30B2081318142812C
:10615000538162177307840795074CF081E090E044
:10616000A0E0B0E080839183A283B383089510827E
:10617000118212821382089588E19EE268E30E94F0
:1061800027184091192E21E030E0241B3109220FFD
:10619000331F220F331FE0911A2EF0911B2EE21BAA
:1061A000F30B208131814281538162177307840789
:1061B00095074CF481E090E0A0E0B0E0808391830B
:1061C000A283B383089510821182128213820895EC
:1061D00088E19EE268E30E9427184091192E21E091
:1061E00030E0241B3109220F331F220F331FE091AF
:1061F0001A2EF0911B2EE21BF30B2081318142817C
:10620000538126173707480759074CF481E090E07F
:10621000A0E0B0E080839183A283B38308951082CD
:1062200011821282138208950F931F9388E19EE2D8
:1062300068E30E9427189B01AC016091192E81E050
:1062400090E0861B9109880F991F880F991F009174
:106250001A2E10911B2E081B190BF80160817181F9
:10626000828193810E947E3EF801608371838283E4
:1062700093831F910F9108950F931F9388E19EE2DE
:1062800068E30E9427189B01AC016091192E81E000
:1062900090E0861B9109880F991F880F991F009124
:1062A0001A2E10911B2E081B190BF80160817181A9
:1062B000828193810E94DF3EF80160837183828333
:1062C00093831F910F91089588E19EE268E30E94F5
:1062D00027184091192E21E030E0241B3109220FAC
:1062E000331F220F331FE0911A2EF0911B2EE21B59
:1062F000F30B2081318142815381261B370B480BE0
:10630000590B2083318342835383089588E19EE2B1
:1063100068E30E9427184091192E21E030E0241BE9
:106320003109220F331F220F331FE0911A2EF091F3
:106330001B2EE21BF30B2081318142815381260FFA
:10634000371F481F591F2083318342835383089589
:1063500088E19EE268E30E9427184091192E21E00F
:1063600030E0241B3109220F331F220F331FE0912D
:106370001A2EF0911B2EE21BF30B208131814281FA
:106380005381262337234823592320833183428393
:106390005383089588E19EE268E30E9427184091A4
:1063A000192E21E030E0241B3109220F331F220F68
:1063B000331FE0911A2EF0911B2EE21BF30B20816C
:1063C000318142815381262B372B482B592B208337
:1063D000318342835383089588E19EE268E30E94FB
:1063E00027184091192E21E030E0241B3109220F9B
:1063F000331F220F331FE0911A2EF0911B2EE21B48
:10640000F30B20813181428153812627372748278A
:1064100059272083318342835383089588E19EE284
:1064200068E30E942718CB010895CF92DF92EF9284
:10643000FF920F931F9388E19EE268E30E94271862
:106440006B017C01C114D104E104F104F9F0209145
:10645000192E81E090E0821B9109880F991F880F07
:10646000991F00911A2E10911B2E081B190BF80171
:106470006081718182819381A70196010E94DF3E34
:10648000F801208331834283538305C08AE18093DE
:106490007A2D0E94E9211F910F91FF90EF90DF90DC
:1064A000CF9008950F931F93682F84E19EE247E1F8
:1064B0000E940D183DC080917A2D8823F1F5E0915E
:1064C000162EF091172EE90FF11D42915291403195
:1064D000A1F1242F30E0207F3070852F90E0807F65
:1064E0009070821793074CF1413169F4503159F49F
:1064F00084E19EE268E30E94FA1784E19EE268E389
:106500000E94FA171AC084E19EE268E30E94FA171B
:10651000082F84E19EE268E30E94FA17182F84E1B5
:106520009EE2602F47E10E940D18812F0E94B62E37
:106530009091152E923008F0BECF1F910F910895C3
:10654000893328F4873360F4813141F409C08A33F8
:1065500039F08A3318F08A57863010F080E00895B9
:1065600081E10E94523281E00895CF93DF93843815
:1065700061F0853820F4833809F081C070C0843917
:1065800079F1843A09F07BC014C0E091862DF09136
:10659000872D818192813396F093872DE093862D0C
:1065A0000F960E94070DFC01408151816281738129
:1065B0006CC0E091862DF091872D418152816381DD
:1065C00074813596F093872DE093862D35978581DC
:1065D0003696E80FF11DF093872DE093862D55C078
:1065E000E091862DF091872D818192813396F093F1
:1065F000872DE093862D0F960E94070DFC01C08128
:10660000D1818091862D9091872D01969093872D31
:106610008093862D0E944D338091862D9091872DF9
:1066200001969093872D8093862D88E19EE268E302
:106630000E942718FB0188819981E817F90720F04B
:1066400089E180937A2D26C0EE0FFF1FEE0FFF1F0A
:10665000EC0FFD1F428153816481758116C0E0916A
:10666000862DF091872D818192813396F093872D2D
:10667000E093862D0E94470EAB01BC0106C088E066
:1066800080937A2D0E94E92105C088E19EE227E1EE
:106690000E944718DF91CF9108951F9380E10E94D7
:1066A00052320E94C126E091862DF091872D808183
:1066B000803141F43196F093872DE093862D0E942E
:1066C0004D3318C087FF07C00E94B53280917A2DE4
:1066D000882339F319C00E94F235182F80917A2D42
:1066E000882391F4812F0E94A032882369F4812F9E
:1066F0000E9452328091862D9091872D0196909321
:10670000872D8093862DCDCF1F910895EF92FF9214
:106710000F931F93CF93DF930E944D332091192E37
:1067200081E090E0821B9109880F991F880F991FC3
:10673000C0911A2ED0911B2EC81BD90BE880F9806E
:106740000A811B81E114F1040105110569F48EE44D
:1067500091E6ACEBB0E08093100390931103A0930B
:106760001203B093130328C06091100370911103BA
:1067700080911203909113032DE036E649E150E039
:106780000E947E3E615A7C408149934C6093100385
:10679000709311038093120390931303A801970140
:1067A0000E94BD3E9B01AC012F5F3F4F4F4F5F4F9B
:1067B000288339834A835B83DF91CF911F910F91A7
:1067C000FF90EF900895AF92BF92CF92DF92EF9239
:1067D000FF920F931F930E944D332091192E81E059
:1067E00090E0821B9109880F991F880F991FE091F3
:1067F0001A2EF0911B2EE81BF90BA080B180C280ED
:10680000D380E12CF12C012DA0E41A2F07C072E0F7
:1068100016950795F794E7947A95D1F7AE14BF04CF
:10682000C006D106A0F320E030E040E050E024C0F4
:10683000D801C701820F931FA41FB51FA816B90660
:10684000CA06DB0670F0A81AB90ACA0ADB0AD80120
:10685000C701880F991FAA1FBB1F280F391F4A1F86
:106860005B1F569547953795279582E016950795B6
:10687000F794E7948A95D1F7E114F1040105110525
:10688000B9F62A153B054C055D0520F42F5F3F4FF7
:106890004F4F5F4F20833183428353831F910F916A
:1068A000FF90EF90DF90CF90BF90AF9008951F932F
:1068B000DF93CF9300D000D0CDB7DEB7182F0E9462
:1068C0004D332091192E81E090E0821B9109880FB1
:1068D000991F880F991FE0911A2EF0911B2EE81B2B
:1068E000F90B6081718182819381123039F014300B
:1068F00071F0113099F40E94DF130BC00E94D21284
:1069000069837A838B839C830E94340D0EC00E941E
:10691000F61269837A838B839C8307C083E080931C
:106920007A2D19821A821B821C8229813A814B811D
:106930005C816091192E81E090E0861B9109880F9F
:10694000991F880F991FE0911A2EF0911B2EE81BBA
:10695000F90B20833183428353830F900F900F9064
:106960000F90CF91DF911F91089584E00E945734DA
:10697000089582E00E945734089581E00E945734C0
:1069800008950E944D332091192E81E090E0821BE2
:106990009109880F991F880F991FE0911A2EF09185
:1069A0001B2EE81BF90BA081B1818D919D910D905B
:1069B000BC91A02D80839183A283B38308950E940C
:1069C0004D332091192E81E090E0821B9109880FB0
:1069D000991F880F991FE0911A2EF0911B2EE81B2A
:1069E000F90BA081B1818D919C91A0E0B0E08083F2
:1069F0009183A283B38308950E944D332091192E71
:106A000081E090E0821B9109880F991F880F991FE0
:106A1000E0911A2EF0911B2EE81BF90BA081B18199
:106A20008C9190E0A0E0B0E080839183A283B38357
:106A300008950E944D3308950E944D332091192EE0
:106A400081E090E0821B9109880F991F880F991FA0
:106A5000E0911A2EF0911B2EE81BF90B8081918199
:106A6000A281B3810097A105B10529F4108211829A
:106A7000128213820895B7FF05C08FEF9FEFAFEF2B
:106A8000BFEF04C081E090E0A0E0B0E0808391839C
:106A9000A283B38308950E944D332091192E81E083
:106AA00090E0821B9109880F991F880F991FE09130
:106AB0001A2EF0911B2EE81BF90B2081318137FF34
:106AC00003C0309521953F4FC901AA2797FDA09596
:106AD000BA2F80839183A283B3830895CF93DF93EA
:106AE000843861F0853820F4833809F06DC05CC0CB
:106AF0008439D1F0843A09F067C014C0E091862D42
:106B0000F091872D818192813396F093872DE093C8
:106B1000862D0F960E94070DAC01662757FD6095E4
:106B2000762F58C08AE351C0E091862DF091872DD1
:106B3000818192813396F093872DE093862D0F9675
:106B40000E94070DFC01C081D1818091862D90911A
:106B5000872D01969093872D8093862D0E944D332B
:106B60008091862D9091872D01969093872D80930B
:106B7000862D88E19EE268E30E942718888199812A
:106B80006817790720F089E180937A2D28C0229632
:106B9000660F771F660F771FC60FD71FAE016627D8
:106BA00057FD6095762F16C0E091862DF091872DC8
:106BB000818192813396F093872DE093862D0E94F8
:106BC000CF0CAB01BC0106C088E080937A2D0E94F7
:106BD000E92105C088E19EE227E10E944718DF9184
:106BE000CF910895863309F071C0E091862DF09120
:106BF000872D3196F093872DE093862D31978181F3
:106C00003396F093872DE093862D33978A30F1F1F8
:106C10008B3098F4853059F1863040F4833021F17F
:106C20008430F8F4823009F041C039C08730B9F1BE
:106C3000873000F18930D1F520C08F3009F18031E3
:106C400038F48D3061F18E3050F58B3079F527C0F6
:106C5000813149F18131B8F08231D9F0833131F598
:106C60001BC00E944B3522C00E94E3331FC00E940C
:106C700086331CC00E941C3519C00E94FC3416C00B
:106C80000E94DF3413C00E94C13410C00E94BD3482
:106C90000DC00E94B9340AC00E94B53407C089E211
:106CA00080937A2D03C083810E946E358091862D5A
:106CB0009091872D01969093872D8093862D0E9429
:106CC000C126E091862DF091872D80810895E09175
:106CD000862DF091872D8081E80FF11DF093872D8F
:106CE000E093862D0895E091862DF091872D808187
:106CF000E80FF11DF093872DE093862D0895A09164
:106D0000862DB091872DFD012191F093872DE09381
:106D1000862D243951F411962D913C91129713969A
:106D2000B093872DA093862D18C0223819F420E047
:106D300030E015C011968D919C911297FD0133960C
:106D4000233831F49C01F093872DE093862D07C002
:106D5000F093872DE093862D9C01215F3F4FC90161
:106D60000895E0915106EE2321F48DE180937A2D70
:106D70000895E150E0935106F0E0EE0FFF1FE45D4F
:106D8000FB4C808191819093872D8093862D08956F
:106D900008950895CF93DF93E0918E2DEE2331F483
:106DA0008FE180937A2D0E94E92124C0C091862D25
:106DB000D091872DF0E0EE0FFF1FEA58FA4F808147
:106DC00091819093872D8093862D0E944D3388E189
:106DD0009EE268E30E9427186115710581059105FF
:106DE00049F4D093872DC093862D80918E2D8150AC
:106DF00080938E2DDF91CF910895CF93DF930E94E2
:106E0000C126C091862DD091872D8091BE05882303
:106E100051F0809172059091730501979093872DA1
:106E20008093862D06C02396D093872DC093862D00
:106E300023970E94C12620915106203121F48CE134
:106E400080937A2D13C0E22FF0E0EE0FFF1FE45D78
:106E5000FB4C8091862D9091872D918380832F5FAD
:106E600020935106D093872DC093862DDF91CF912B
:106E700008950E94340D81E08093772D1092922D19
:106E80001092912D809172059091730501979093C6
:106E9000872D8093862D0895CF93DF9320918E2D9B
:106EA000203131F48EE180937A2D0E94E92141C096
:106EB000E22FF0E0EE0FFF1FE858FA4F8091862D89
:106EC0009091872D918380832F5F20938E2DC1E039
:106ED000D0E0E0917605F0917705F093872DE0936F
:106EE000862D309731F18091720590917305E817E6
:106EF000F90719F40E9439371CC082819F01280FBD
:106F0000311D30937705209376053396F093872DC6
:106F1000E093862D0E94C126E091862DF091872D69
:106F2000E081E93111F42196D4CFEA3191F621972D
:106F300081F6DF91CF91089583EF98E10E947F0D54
:106F40006091912D7091922D80E090E00E946F21D0
:106F50001092772D80917605909177059093AB33C1
:106F60008093AA331092922D1092912D80917205E8
:106F70009091730501979093872D8093862D0895A6
:106F80000E94C126E091862DF091872D21813281CA
:106F90003396F093872DE093862D5091BE055523AF
:106FA00041F08091720590917305909377058093DD
:106FB0007605E0917605F091770560917205709104
:106FC0007305E617F70721F4E0918A2DF0918B2DD8
:106FD000808191812817390720F4E0918A2DF09162
:106FE0008B2D8081918182179307B1F4F093872DC7
:106FF000E093862D552341F01092BE0581E08093E9
:107000004E060E94A42808953396F093872DE093AE
:10701000862D0E94C126089542812817390728F03D
:10702000E40FF11DE617F707E1F68BE180937A2D67
:107030000895AF92BF92CF92DF92EF92FF920F939B
:107040001F93CF93DF93E091862DF091872D1081D0
:10705000103731F0133721F0143711F000E00DC074
:107060003196F093872DE093862D0E94C126E09102
:10707000862DF091872D012F10810E947F367C0193
:10708000143919F0C0E0D0E034C08091862D909181
:10709000872D01969093872D8093862D0E944D33E6
:1070A0008091862D9091872D01969093872D8093C6
:1070B000862D80917A2D882309F082C0C7010E9415
:1070C000070DFC01C081D18188E19EE268E30E9446
:1070D0002718888199816817790720F089E18093C2
:1070E0007A2D6EC02296660F771F660F771FC60F28
:1070F000D71F0E94C1268091862D9091872D0196E1
:107100009093872D8093862D0E944D3380917A2D08
:10711000882309F055C088E19EE268E30E942718A1
:107120005B016C01133831F4C701B601A5010E945F
:10713000060E46C0143929F4688379838A839B83B9
:107140003FC0C7010E94070DFC010023D9F0208138
:10715000318142815381003749F4CA01AA27BB27F4
:10716000F9010BB68BBFA0820BBE2AC0043779F49D
:10717000CA01AA27BB27F9010BB68BBFA192B08227
:107180000BBE1EC09C01442737FD4095542FCA01F9
:10719000AA27BB27F9010BB68BBFA192B0820BBE09
:1071A0002E5F3F4F4F4F5F4F7A0100271127C601D7
:1071B000AA27BB27F9010BB6EBBE819390830BBEC8
:1071C000DF91CF911F910F91FF90EF90DF90CF90C3
:1071D000BF90AF9008958FEF80936B050895109244
:1071E0006B05089508958091862D9091872D0396C3
:1071F0009093872D8093862D0E944D338091862D0C
:107200009091872D01969093872D8093862D0895D8
:107210001F93182F82958F708A3008F0895F805DE8
:107220000E949E0D812F8F708A3008F0895F805DEB
:107230000E949E0D1F910895EF92FF920F931F934E
:107240000E94F33888E19EE268E30E9427187B01E0
:107250008C01892F9927AA27BB270E940839C801CA
:10726000AA27BB270E940839BB27A12F902F8F2D5B
:107270000E9408398E2D0E9408391F910F91FF90AE
:10728000EF900895EF92FF920F931F930E94F338AF
:1072900088E19EE268E30E9427187B018C01BB27EE
:1072A000A92F982F872F0E9408398E2D0E94083908
:1072B0001F910F91FF90EF9008950E94F33888E19D
:1072C0009EE268E30E942718862F0E9408390895DD
:1072D0000E94F33888E19EE268E30E942718862F17
:1072E0000E949E0D08950E94F33888E19EE268E3B3
:1072F0000E94271889E00E949E0D0895EF92FF9248
:107300000F931F930E94C126E091862DF091872D47
:10731000E08110E07BC0EB37B1F1EC3720F4E633CD
:1073200009F05FC03BC0EC3759F1E23A09F059C0AF
:10733000E091862DF091872D6181E62EFF2400E0FB
:1073400010E08EEF9FEFAFEFBFEFE80EF91E0A1FC0
:107350001B1F3396F093872DE093862DCF01B70145
:107360000E94C83CB7016F5F7F4F8091862D90913E
:10737000872D860F971F9093872D8093862D23C08E
:1073800089E00E949E0D8091862D9091872D019617
:107390009093872D8093862D11E031C0E091862D4A
:1073A000F091872D81818B3099F08C3028F48230D8
:1073B00061F08730B1F405C08D3069F08E3089F40A
:1073C0000DC00E94733910E01AC00E94683928C0AD
:1073D0000E941C3925C00E945D3922C00E9442399A
:1073E0001FC00E944D3380917A2D8823E9F488E1F3
:1073F0009EE268E30E9427180E946F2111C00E943C
:10740000C126E091862DF091872DE081ED3719F0AE
:10741000EA3709F080CF112339F40E94340D04C0FB
:1074200080E20E949E0DCFCF1F910F91FF90EF90B1
:107430000895EF92FF920F931F93CF93DF93E09005
:10744000B705F090B8050E94C126E091862DF09115
:10745000872D808184FD02C081E22FC081819281CD
:107460000F960E94070DEC018091862D9091872D3B
:1074700004969093872D8093862D0E944D338091A2
:10748000862D9091872D01969093872D8093862D40
:1074900088819981AA81BB810097A105B10509F076
:1074A00047C00091B7051091B80588E19EE268E3F6
:1074B0000E94271877FF04C087E280937A2D47C087
:1074C0004091B7055091B805198308831B821A8231
:1074D0006F5F7F4FF801718360834E5F5F4FCB0119
:1074E000880F991F880F991F840F951F4250504095
:1074F0009093B8058093B70520919E3330919F33C8
:107500002817390720F0FA0180E090E00EC089E0EA
:1075100080937A2DF092B805E092B70518C01282D8
:107520001382148215820196349686179707B8F352
:107530000E94C126E091862DF091872D80818D37A4
:1075400031F03196F093872DE093862D78CFDF913F
:10755000CF911F910F91FF90EF9008950895089596
:107560000895089508950895089508950895089533
:1075700008958091BE05882329F083E380937A2DB6
:107580000E94E9210895CF93DF93C091862DD09179
:10759000872D80918A2D90918B2D9093872D8093AC
:1075A000862D90935F0680935E06E091862DF09184
:1075B000872D82819F01280F311D30935F06209314
:1075C0005E063396F093872DE093862D0E94C126A8
:1075D000E091862DF091872D80818C3051F4329688
:1075E000F0935F06E0935E06D093872DC093862DBF
:1075F0001AC020915E0630915F06809172059091CD
:1076000073052817390751F4D093872DC093862D21
:1076100086E280937A2D0E94E92105C03093872D60
:107620002093862DC2CFDF91CF910895CF93DF9322
:10763000C091862DD091872D80915E0690915F0636
:107640009093872D8093862D8091862D9091872D04
:1076500003969093872D8093862D0E94C126E091FA
:10766000862DF091872D80818C3051F43396F093E4
:107670005F06E0935E06D093872DC093862D1BC0D6
:10768000E0915E06F0915F0680917205909173051E
:10769000E817F90741F4D093872DC093862D86E231
:1076A00080937A2D08C08281E80FF11DF0935F0668
:1076B000E0935E06C9CFDF91CF910895CF92DF921C
:1076C000EF92FF920F931F930E94C1260E947F3674
:1076D0008C010E94A60DC82EC8010E94070DFC0156
:1076E000DD24EE24FF24C082D182E282F3821F9146
:1076F0000F91FF90EF90DF90CF900895CF93DF939D
:107700000E94C1260E947F369C0190916C058EE0FC
:10771000989FE0011124CD54DA4F88819981281770
:10772000390731F084E280937A2D0E94E92145C027
:10773000C9010E94070DFC012081318142815381E2
:107740008A819B81AC81BD81280F391F4A1F5B1F35
:1077500020833183428353838A819B81AC81BD81A5
:10776000B7FF0AC08E819F81A885B9852817390780
:107770004A075B07B4F40DC00097A105B10589F075
:107780008E819F81A885B98582179307A407B507C5
:1077900044F480916C05815080936C050E94C12651
:1077A0000CC08A859B859093872D8093862D8C8530
:1077B0009D859093922D8093912DDF91CF91089587
:1077C000DF92EF92FF920F931F93D82E8091862D18
:1077D0009091872D01969093872D8093862D0E94FE
:1077E000C1260E944D330E94C1268091862D909122
:1077F000872D01969093872D8093862D0E94C12618
:107800008091862D9091872D01969093872D80935E
:10781000862D0E944D3388E19EE268E30E9427187E
:107820007B018C0188E19EE268E30E94271822E038
:10783000D216A1F034E0D316F9F041E0D41611F5D8
:1078400080E090E02FEF30E040E050E0E222F322D1
:10785000042315234E2D0E947E1714C080E090E073
:107860002FEF3FEF40E050E0E222F3220423152304
:10787000A7010E943D1706C080E090E0A801970193
:107880000E9456171F910F91FF90EF90DF9008957F
:1078900084E00E94E03B089582E00E94E03B08956E
:1078A00081E00E94E03B08950E944D330E94C12672
:1078B0008091862D9091872D01969093872D8093AE
:1078C000862D0E94C12688E19EE268E30E94271867
:1078D0009B01AC0180917A2D8823C1F5E091862D22
:1078E000F091872D232B31F08081883A79F50E9421
:1078F000C03708958081883A79F43396F093872DC4
:10790000E093862D0E94C126E091862DF091872D6F
:1079100080818933D9F40AC08091760590917705EA
:1079200001979093872D8093862D08953196F0933B
:10793000872DE093862D0E94C126E091862DF0913F
:10794000872D8081883A11F40E94C03708951F93D3
:10795000E0918F2DF091902D80818D3211F010E00B
:1079600006C03196F093902DE0938F2D11E00E9488
:107970009A1E9B01AC01112339F05095409530952A
:1079800021953F4F4F4F5F4FB901CA011F91089595
:107990000F931F93CF93DF938C01EB0106C0F80187
:1079A00081918F010E94430D21972097C1F7DF91AC
:1079B000CF911F910F910895EF92FF920F931F9314
:1079C000E0918F2DF091902D8081843241F4319699
:1079D000F093902DE0938F2D0E943E1F02C00E94D5
:1079E000A73C7B018C010E946718E0918F2DF091DC
:1079F000902D80818D3071F08C3231F43196F0937E
:107A0000902DE0938F2D06C085E180937A2D0E9402
:107A1000E92109C00E947F360E94070DFC01E08227
:107A2000F182028313831F910F91FF90EF900895CD
:107A30000E946718E0918F2DF091902D80818D30FC
:107A4000C9F00E94DC3C80917A2D882399F40E9431
:107A5000C126E091862DF091872D80818D3769F0C8
:107A60008A3759F03196F093872DE093862D0E9446
:107A7000C126DECF21E030E002C020E030E0C901C5
:107A8000089580915E0690915F06892B21F40E94F3
:107A9000C33A0E94163B80915E0690915F069093D8
:107AA000902D80938F2D0E94C1260E94183D209119
:107AB0008F2D3091902D019769F42E5F3F4F3093B9
:107AC0005F0620935E060E94163B80917A2D8823E4
:107AD00011F304C030935F0620935E060895EF9281
:107AE000FF920F931F930E94C126E091862DF09183
:107AF000872D8081823A01F5018110E0025010400B
:107B000083E0E82EF12CEE0EFF1EC701B8010E94A3
:107B1000C83C0F5F1F4FE00EF11EF092872DE092E0
:107B2000862D0E94C1268091862D9091872D0196E9
:107B30009093872D8093862D0E94C1268FE30E940B
:107B40009E0D80E20E949E0D0E94C71A0E94340D75
:107B50000E940927882321F40E94183D892B71F780
:107B600010924C341F910F91FF90EF9008950F9356
:107B70001F9380916C058A3031F483E280937A2DD3
:107B80000E94E921B8C00E94C1260091862D109163
:107B9000872D0E947F3640916C05242F30E0220F04
:107BA000331FF90173E0EE0FFF1F7A95E1F7E21B37
:107BB000F30BEF53FA4F91838083842F90E0880F6B
:107BC000991FFC0153E0EE0FFF1F5A95E1F7E81BE8
:107BD000F90BEF53FA4F8091912D9091922D95874B
:107BE00084871093872D0093862D0E9419380E9458
:107BF000C1268091862D9091872D01969093872D97
:107C00008093862D0E94C1260E944D3310916C05F1
:107C100088E19EE268E30E942718212F30E0220FBE
:107C2000331FF90103E0EE0FFF1F0A95E1F7E21B96
:107C3000F30BEF53FA4F66837783808791878091A8
:107C40006C0590E0FC0113E0EE0FFF1F1A95E1F7C1
:107C5000E81BF90BEE0FFF1FED53FA4F81E090E0A8
:107C6000A0E0B0E080839183A283B3830E94C12609
:107C7000E091862DF091872D80818A3319F5319618
:107C8000F093872DE093862D0E94C1260E944D33EC
:107C900000916C0510E088E19EE268E30E942718DD
:107CA000F801A3E0EE0FFF1FAA95E1F7E01BF10B2F
:107CB000EE0FFF1FED53FA4F60837183828393832E
:107CC0000E94C12620916C05822F90E0880F991F99
:107CD000FC0133E0EE0FFF1F3A95E1F7E81BF90BCB
:107CE000EF53FA4F8091862D9091872D938782874D
:107CF0002F5F20936C051F910F910895629FD00113
:107D0000739FF001829FE00DF11D649FE00DF11D56
:107D1000929FF00D839FF00D749FF00D659FF00D05
:107D20009927729FB00DE11DF91F639FB00DE11DF2
:107D3000F91FBD01CF0111240895991B79E004C0FA
:107D4000991F961708F0961B881F7A95C9F780959A
:107D50000895AA1BBB1B51E107C0AA1FBB1FA61792
:107D6000B70710F0A61BB70B881F991F5A95A9F7E4
:107D700080959095BC01CD010895A1E21A2EAA1B11
:107D8000BB1BFD010DC0AA1FBB1FEE1FFF1FA217CB
:107D9000B307E407F50720F0A21BB30BE40BF50BC8
:107DA000661F771F881F991F1A9469F76095709551
:107DB000809590959B01AC01BD01CF01089597FB83
:107DC000092E05260ED057FD04D0D7DF0AD0001C9F
:107DD00038F450954095309521953F4F4F4F5F4F68
:107DE0000895F6F790958095709561957F4F8F4F28
:107DF0009F4F089585FD5AC08062911157C08156EA
:107E00008A51E0F70895911151C080538A5028F0AB
:107E1000865C806281568650B8F708959111089566
:107E200081548A5108F4805E855A0895911108950D
:107E300081568A5108F4805285580895FB01DC016F
:107E400005900D920020E1F70895FC0105900020B7
:107E5000E9F7809590958E0F9F1F0895FB01DC0137
:107E60000D900020E9F7119701900D920020E1F7A5
:107E70000895FB01DC0101900D920020E1F70895C7
:107E8000F999FECF92BD81BDF89A992780B50895E2
:107E9000262FF999FECF1FBA92BD81BD20BD0FB626
:107EA000F894FA9AF99A0FBE0196089599278827AF
:067EB0000895F894FFCFD5
:107EB600010102014201430183018401646174618D
:107EC600006C6574007265616400726573746F722C
:107ED6006500676F73756200676F746F006F6E0081
:107EE60072657475726E00696600696E70757400ED
:107EF6007072696E7400666F72006E6578740073D6
:107F0600746F7000656E64776800656E64007265F4
:107F16006D0064696D0074726F6E0074726F6666D0
:107F2600007768696C650065657031360065657057
:107F360033320065657000696E62797465003F00D2
:107F46002700656C7365003C3D003E3D003C3E00ED
:107F56003C003E003D00414E44004F5200454F520A
:107F6600002B002D002A002F006D6F64005E00407C
:107F76003136004033320040006E6F7400746F007B
:107F860053544550007468656E00656C7365004710
:107F96004F544F00474F5355420043485224006107
:107FA6006273007371727400524E440053474E0060
:107FB6005441420068657834006865783200686527
:107FC60078007065656B3136007065656B3332001D
:107FD6007065656B006164647200656570313600BA
:107FE6006565703332006565700074696D652400DF
:107FF600706F727473004C697374206F6620706FB3
:10800600727473202D2D00200076617273004C6906
:108016007374206F66207661726961626C65732085
:108026002D2D002020202000280029002020006679
:10803600696C657300556E6B6E6F776E204C495395
:108046005420746F7069632E202054727920276C37
:1080560069737420706F72747327206F7220276C97
:10806600697374207661727327206F7220276C699A
:1080760073742066696C6573272E006D6F6E006CD5
:108086006973740072756E006E657700636F6E7447
:1080960000636C6561720066726565006C6F616491
:1080A6000073617665006175746F7374006F666640
:1080B60000656500666C3000666C3100666C3200E7
:0480C6004E61BC004B
:020000021000EC
:10FC0000AF92BF92CF92DF92EF92FF920F931F932A
:10FC1000CF93DF937B018C016A01AFB6F894F99919
:10FC2000FECF07B600FCFDCF83E0F70100935B0039
:10FC300080935700E89507B600FCFDCF40E050E008
:10FC400060E070E0BB24B394F6018081D181C0E014
:10FC50009E01280F311D82E090E0C80ED91EDB0105
:10FC6000CA018E0D9F1DA01FB11F0901FC01A093A9
:10FC70005B00B0925700E89511244E5F5F4F6F4FC5
:10FC80007F4F403091E0590790E0690790E0790795
:10FC9000D9F685E0F70100935B0080935700E89563
:10FCA00007B600FCFDCF81E180935700E895AFBE19
:10FCB000DF91CF911F910F91FF90EF90DF90CF9048
:06FCC000BF90AF90089513
:00000001FF
